:04000000E1EF3FF0FD
:1000080000C016F001C015F0E1CF17F0E2CF18F0EC
:100018009DAA68D09EAA66D0AECFFFF0ABA411D03F
:10002800AB9E010E01010325006E000E0421016E36
:1000380000C003F101C004F1AB8EAECFFFF00001A8
:10004800FF6BABA211D0AB98AB88010E010105255F
:10005800006E000E0621016E00C005F101C006F118
:10006800AECFFFF00001FF6B0001FF510D0A11E058
:10007800980E1924E16E000E1A20E26EFFC0E6FF0A
:10008800194A1A2A19C096F01AC097F0FA6BFB6B36
:100098000DD0980E1924E16E000E1A20E26EE66A61
:1000A800010EFA6F000EFB6F196A1A6A800E006E55
:1000B800800E1A18005C02E11950170812E2020EAD
:1000C800FA6F000EFB6F9D9A010E195C006E000E10
:1000D8001A58016E980E0024E16E000E0120E26E9F
:1000E800E66A9E9A9DA022D09EA020D0010E010112
:1000F8002325006E000E2421016E00C023F101C0EB
:1001080024F1800E2419006E800E005C02E1080EB6
:10011800235D07E3236B246B010E1F6F000E206F16
:100128009D900B0ECF6EDB0ECE6E9E9016C000F02B
:0E01380015C001F017C0E1FF18C0E2FF110072
:100146000B820BAEADEF00F0036802680168006831
:080156000A360232FF0E12000E
:0E015E00026A016A006A086A036A000E120053
:10016C000B840BAEC1EF00F0010E036E026A016A44
:0A017C00006A0A360232FF0E12007C
:080186000AAE029E000E1200F9
:10018E000CB009EF01F00CA2AFEF01F00E6A000EF9
:10019E00026420EF01F0F00E0214D8A4EBEF00F091
:1001AE00023A01380F0B02260138F00B016E0038AF
:1001BE000F0B01260038F00B006E08380F0B0026CF
:1001CE000838F00B086E0E84D89002BE04EF01F0D2
:1001DE0008360036013602360E2A02BE04EF01F052
:1001EE0008360036013602360E2A02BE04EF01F042
:1001FE0008360036013602360E2A0E500364A5EF7D
:10020E0001F0035E0BBC08AEAAEF01F0D880800EA1
:10021E0008640030000E002201220222D8A0AAEFAC
:10022E0001F0023201320032034AAFEF01F0AAEFC1
:10023E0001F001C002F000C001F008C000F0086A31
:10024E00000E0E86026457EF01F0F00E0214D8A4D1
:10025E003FEF01F0023A01380F0B02260138F00B86
:10026E00016E00380F0B01260038F00B006E0E8465
:10027E00D89002BE04EF01F00036013602360E2A87
:10028E0002BE04EF01F00036013602360E2A02BE1F
:10029E0004EF01F00036013602360E2A04EF01F0AB
:1002AE0001C002F000C001F0006A000E0E960E882A
:1002BE00026484EF01F0F00E0214D8A46FEF01F087
:1002CE00023A01380F0B02260138F00B016E0E8434
:1002DE00D89002BE04EF01F0013602360E2A02BE9D
:1002EE0004EF01F0013602360E2A02BE04EF01F0D1
:1002FE00013602360E2A04EF01F001C002F0016A47
:10030E00000E0E860264B4EF01F0F00E0214D8A4B3
:10031E0093EF01F0023A0E84D89002BE04EF01F082
:10032E0002360E2A02BE04EF01F002360E2A02BE7B
:10033E0004EF01F002360E2A04EF01F0010E0C6EEE
:10034E000EDFB7EF01F0020E0C6E16DFB7EF01F005
:10035E00040E0C6EF1DEB7EF01F0080E0C6EF8DE37
:02036E0012007B
:080370000B6A0B86FF0E120060
:10037800086A096A000E0762036441EF02F002503E
:1003880006180A6E075003267E0ED8A0D2EF01F099
:10039800035ED8B045EF02F0D6EF01F0035ED8A0B7
:1003A80049EF02F0028E068E02C00EF001C00BF07B
:1003B80000C00DF000500402F4CF0CF0015005020B
:1003C800F4CF00F0F3CF08F00402F3500C26F450F9
:1003D8000822000E00220D500502F3500C26F4509E
:1003E8000822000E002202500402F3500826F4509E
:1003F800002202500502016A000E0122F350002675
:10040800F45001220D500602F3500826F450002241
:10041800026A000E012202220B500602F350002647
:10042800F4500122000E02220E500602F35001265B
:10043800F450022202BE29EF02F0083600360136D7
:1004480002360306D8B449EF02F03CEF02F0D88038
:10045800800E08640030000E002201220222D8A07B
:100468003CEF02F0023201320032034A45EF02F05B
:100478000AAE029E000E4BEF02F0010E6CDE4BEF4F
:1004880002F0020E5CDE4BEF02F0040E6BDE12008F
:100498000D6A086A0050D8B4000C04180A6E0ABE27
:1004A8000D1E0B6A04AE02D0041E042A00AE02D050
:1004B800001E002A005004100A6E0ABE1FD0045005
:1004C800085E003600340836045008260036060E4A
:1004D8000C6E00340836045000B0085E00A00826F0
:1004E80000360C2EF6D700A008260BB015D00DAE9E
:1004F800000C001E002A081E082A000C04AE09D0B1
:1005080000BE04D00050086E006AF1D7006A002AC5
:10051800000C001E0B2AD3D7082A0450085CD8A464
:0E052800E6D7086A002A00AEE2D7FF0C1200E8
:10053600086A080E0C6E003408360450085ED8B0FF
:0E05460002D00826D89000360C2EF5D71200F1
:10055400025006180E6E086A096A0B6A0350076493
:100564009DEF03F006500A6E068E028E03500B6E4A
:100574000750036E000E0B64EDEF02F00B50075EA4
:10058400D8B48EEF03F0070E07645CEF03F0075E48
:1005940000C008F001C000F002C001F0026A074E7A
:1005A4008EEF03F0076431EF03F0075E00C008F03C
:1005B40001C000F0016A074E8EEF03F007640FEFED
:1005C40003F0075E00C008F0006A074E8EEF03F0E8
:1005D4000764F6EF02F00AC002F005C001F004C09F
:1005E40000F0086AB8EF04F0030E076401EF03F0AB
:1005F400075E08380F0B086E074E8EEF03F0D89095
:100604000832074E8EEF03F0D8900832074E8EEF73
:1006140003F0D89008328EEF03F0030E076420EF46
:1006240003F0075E08380F0B086E0038F00B08263D
:1006340000380F0B006E074E8EEF03F0D890003297
:100644000832074E8EEF03F0D89000320832074E7E
:100654008EEF03F0D890003208328EEF03F0030ED1
:10066400076448EF03F0075E08380F0B086E003884
:10067400F00B082600380F0B006E0138F00B002633
:1006840001380F0B016E074E8EEF03F0D890013244
:1006940000320832074E8EEF03F0D8900132003258
:1006A4000832074E8EEF03F0D89001320032083240
:1006B4008EEF03F0030E076479EF03F0075E08384A
:1006C4000F0B086E0038F00B082600380F0B006E75
:1006D4000138F00B002601380F0B016E0238F00BC5
:1006E400012602380F0B026E074E8EEF03F0D890EE
:1006F4000232013200320832074E8EEF03F0D890F6
:100704000232013200320832074E8EEF03F0D890E5
:100714000232013200320832096A000E0EAE82EF54
:1007240004F0081E001E011E021E082A00220122D7
:10073400022282EF04F00750D8A4A3EF03F0B8EF2D
:1007440004F0096A02C00AF0028E068E0750035CA8
:10075400076ED8B475EF04F0070E076443EF04F096
:10076400075E0450096E0550046E0650056E066A55
:10077400074E75EF04F0070E076418EF04F0075EE8
:100784000450096E0550046E056A074E75EF04F0B7
:10079400070E0764F6EF03F0075E0450096E046A5F
:1007A400074E75EF04F0070E0764DDEF03F00AC08F
:1007B40002F0B8EF04F0030E0764E8EF03F0075EFD
:1007C40009380F0B096E074E75EF04F0D890093203
:1007D400074E75EF04F0D8900932074E75EF04F018
:1007E400D890093275EF04F0030E076407EF04F0A4
:1007F400075E09380F0B096E0438F00B092604381C
:100804000F0B046E074E75EF04F0D89004320932D2
:10081400074E75EF04F0D89004320932074E75EF95
:1008240004F0D8900432093275EF04F0030E076423
:100834002FEF04F0075E09380F0B096E0438F00B34
:10084400092604380F0B046E0538F00B042605380E
:100854000F0B056E074E75EF04F0D8900532043285
:100864000932074E75EF04F0D8900532043209328C
:10087400074E75EF04F0D89005320432093275EF53
:1008840004F0030E076460EF04F0075E09380F0BF1
:10089400096E0438F00B092604380F0B046E053872
:1008A400F00B042605380F0B056E0638F00B0526F1
:1008B40006380F0B066E074E75EF04F0D89006321B
:1008C400053204320932074E75EF04F0D89006322F
:1008D400053204320932074E75EF04F0D89006321F
:1008E400053204320932086A000E0EAE82EF04F0BB
:1008F400091E041E051E061E092A042205220622BC
:1009040009500826045000220550012206500222F4
:100914000EBE99EF04F0D8A0A8EF04F00232013221
:1009240000320832033EA8EF04F0B2EF04F0D8B06E
:10093400ADEF04F0000E081E001E011E021E082A60
:100944000022012202220A7EADEF04F0010E0C6E99
:100954001CDCBAEF04F0020E0C6E17DCBAEF04F0E4
:10096400040E0C6EA3EC00F0BAEF04F0000E0C6E53
:0209740012006F
:100976000B800BAEC7EF04F0026A0AAEFF0E026EE2
:0C098600016E006E0A360232FF0E1200F5
:0E099200ACB202D00000FCD7A7C1ADFF12002E
:1009A0000134083609360450085E0550D8A0053CCD
:1009B000095E003601360F0E0C6E0134083609361A
:1009C000045000A006D0085E0550D8A0053C095E82
:1009D00005D008260550D8B0053C0926003601365A
:1009E0000C2EEBD700B006D0045008260550D8B026
:0809F000053C0926000012007D
:1009F8000B6A0A6A096A086A0E6A033408360450E0
:100A0800085E0550D8A0053C095E0650D8A0063CF3
:100A18000A5E0750D8A0073C0B5EE86AD8A0010E12
:100A28000E5E0336070E0C6E0334083609360A3696
:100A38000B360E36045003A012D0085E0550D8A01D
:100A4800053C095E0650D8A0063C0A5E0750D8A0AF
:100A5800073C0B5EE86AD8A0010E0E5E11D008268E
:100A68000550D8B0053C09260650D8B0063C0A26E1
:100A78000750D8B0073C0B26E86AD8B0010E0E26FE
:100A880003360C2ED1D70234083609360A360B360F
:100A98000E36045003A012D0085E0550D8A0053CBD
:100AA800095E0650D8A0063C0A5E0750D8A0073C4D
:100AB8000B5EE86AD8A0010E0E5E11D0082605501C
:100AC800D8B0053C09260650D8B0063C0A2607507F
:100AD800D8B0073C0B26E86AD8B0010E0E260236BD
:100AE800070E0C6E0234083609360A360B360E36F7
:100AF800045002A012D0085E0550D8A0053C095E3B
:100B08000650D8A0063C0A5E0750D8A0073C0B5EEA
:100B1800E86AD8A0010E0E5E11D008260550D8B09C
:100B2800053C09260650D8B0063C0A260750D8B01E
:100B3800073C0B26E86AD8B0010E0E2602360C2EAA
:100B4800D1D70134083609360A360B360E3604502A
:100B580002A012D0085E0550D8A0053C095E0650D8
:100B6800D8A0063C0A5E0750D8A0073C0B5EE86A8E
:100B7800D8A0010E0E5E11D008260550D8B0053C4D
:100B880009260650D8B0063C0A260750D8B0073CBC
:100B98000B26E86AD8B0010E0E260136070E0C6E39
:100BA8000134083609360A360B360E36045001A0D1
:100BB80012D0085E0550D8A0053C095E0650D8A0A2
:100BC800063C0A5E0750D8A0073C0B5EE86AD8A02E
:100BD800010E0E5E11D008260550D8B0053C092636
:100BE8000650D8B0063C0A260750D8B0073C0B265A
:100BF800E86AD8B0010E0E2601360C2ED1D7003483
:100C0800083609360A360B360E36045001A012D0C3
:100C1800085E0550D8A0053C095E0650D8A0063CE1
:100C28000A5E0750D8A0073C0B5EE86AD8A0010E00
:100C38000E5E11D008260550D8B0053C092606508E
:100C4800D8B0063C0A260750D8B0073C0B26E86AFD
:100C5800D8B0010E0E260036070E0C6E003408368A
:100C680009360A360B360E36045000A012D0085E3C
:100C78000550D8A0053C095E0650D8A0063C0A5E7F
:100C88000750D8A0073C0B5EE86AD8A0010E0E5E9C
:100C980011D008260550D8B0053C09260650D8B012
:100CA800063C0A260750D8B0073C0B26E86AD8B09D
:100CB800010E0E2600360C2ED1D700B00ED00450EF
:100CC80008260550D8B0053C09260650D8B0063C81
:0C0CD8000A260750D8B0073C0B2612007B
:100CE4000B6A0A6A096A00500402F4CF09F0F3CFD0
:100CF40008F001500502F4CF0BF0F3CF0AF00050D6
:100D04000502F3500926F4500A22E86A0B22015026
:100D14000402F3500926F4500A22E86A0B2208C0A0
:100D240000F009C001F00AC002F00BC003F0120089
:100D34000A6A0350D8A40A800750D8A40A820A5029
:100D4400D8B4FDEF06F0030AD8B4B6EF06F00AB043
:100D5400B1EF06F006AEFBEF06F0F9EF06F002AED7
:100D6400F9EF06F0FBEF06F00250800B0A6E029ECC
:100D74000650800B069E0A18D8B4C7EF06F00A5036
:100D8400D8B4F9EF06F0FBEF06F00750035CD8B4D3
:100D9400D1EF06F0D8A0EDEF06F0F3EF06F0065021
:100DA400025CD8B4DBEF06F0D8A0EDEF06F0F3EF69
:100DB40006F00550015CD8B4E5EF06F0D8A0EDEFDD
:100DC40006F0F3EF06F00450005CD8B4FDEF06F033
:100DD400D8B0F3EF06F00A52D8B4FBEF06F0F9EFFF
:100DE40006F00A52D8B4F9EF06F0FBEF06F0D8800B
:0E0DF4001200D8901200D880D884120012008D
:100E02000B6A0C6A086A0350D8B485EF07F002C077
:100E12000AF0028E9E0E035E03AE75EF07F0036CBE
:100E2200080E035CD8A042EF07F0036E083600C03C
:100E320008F001C000F002C001F0026A080E035C73
:100E4200D8A042EF07F0036E083600C008F001C0D8
:100E520000F0016A080E035CD8A042EF07F0036EAF
:100E6200083600C008F0006A080E035CD8A042EF02
:100E720007F0036E0836086A0350D8A4D8904EEFE4
:100E820007F00350D8B44EEF07F0D8900232013287
:100E920000320832032E46EF07F00BBC08A05FEFCA
:100EA20007F0D8A05FEF07F0082AD8B4002AD8B418
:100EB200012AD8B4022A02BE89EF07F00AAE85EFF2
:100EC20007F0021E011E001E081E082AD8B4002ABE
:100ED200D8B4012AD8B4022A85EF07F0026A016A5F
:100EE200006A086A85EF07F00B800BAE8FEF07F000
:100EF200026A0AAE8FEF07F0026E016E006E086E94
:100F02000A3602328FEF07F00C6A000E90EF07F0FC
:100F1200010E0C6E000E2EDD90EF07F0FF0E025058
:100F2200036E0150026E0050016E0850006E1200F6
:100F32000101A251390806E3300EA25D03E3010E5E
:080F4200006E01D0006A1200EC
:100F4A006E0E0101A25DD8A0CAD0640E046EA2C1C1
:100F5A0000F09BEC02F0120E0024056E066A000EE9
:100F6A00062205C000F006C001F0000E06BEFF0E04
:100F7A00026E036E003600900136023603360036E2
:100F8A000090013602360336D10E0024F66E8A0E20
:100F9A000120F76E000E0220F86E0900F5CF00F06E
:100FAA000900F5CF01F00900F5CF02F00900F5CFED
:100FBA0003F0000E046E000E056E000E066E7E0E25
:100FCA00076EBCEC01F000C0A3F101C0A4F102C09D
:100FDA00A5F103C0A6F1640E046EA2C100F09BEC59
:100FEA0002F008C000F00A0E046E9BEC02F0090E33
:100FFA000024056E066A000E062205C000F006C02F
:10100A0001F0000E06BEFF0E026E036E003600905F
:10101A0001360236033600360090013602360336B0
:10102A00D10E0024F66E8A0E0120F76E000E022001
:10103A00F86E0900F5CF00F00900F5CF01F00900BC
:10104A00F5CF02F00900F5CF03F0A3C104F0A4C163
:10105A0005F0A5C106F0A6C107F0BCEC01F000C07E
:10106A00A3F101C0A4F102C0A5F103C0A6F10A0EC2
:10107A00046EA2C100F09BEC02F008C000F000C0B0
:10108A0001F0000E026E036E046E01360190023604
:10109A000336043601360190023603360436D10E81
:1010AA000124F66E8A0E0220F76E000E0320F86EF7
:1010BA000900F5CF00F00900F5CF01F00900F5CFDE
:1010CA0002F00900F5CF03F0A3C104F0A4C105F0B2
:1010DA00A5C106F0A6C107F0BCEC01F0B1D0A2513F
:1010EA000A08D8B07ED00A0E046EA2C100F09BECAA
:1010FA0002F0090E0024056E066A000E062205C0DB
:10110A0000F006C001F0000E06BEFF0E026E036E6E
:10111A00003600900136023603360036009001365A
:10112A0002360336D10E0024F66E8A0E0120F76EBF
:10113A00000E0220F86E0900F5CF00F00900F5CF85
:10114A0001F00900F5CF02F00900F5CF03F0000E17
:10115A00046E000E056E000E066E7E0E076EBCEC67
:10116A0001F000C0A3F101C0A4F102C0A5F103C0BF
:10117A00A6F10A0E046EA2C100F09BEC02F008C0B0
:10118A0000F000C001F0000E026E036E046E01361C
:10119A0001900236033604360136019002360336D0
:1011AA000436D10E0124F66E8A0E0220F76E000E66
:1011BA000320F86E0900F5CF00F00900F5CF01F021
:1011CA000900F5CF02F00900F5CF03F0A3C104F03E
:1011DA00A4C105F0A5C106F0A6C107F0BCEC01F058
:1011EA002FD0A2C100F0000E016E026E036E00360F
:1011FA000090013602360336003600900136023678
:10120A000336D10E0024F66E8A0E0120F76E000E08
:10121A000220F86E0900F5CF00F00900F5CF01F0C1
:10122A000900F5CF02F00900F5CF03F0000E046EB5
:10123A00000E056E000E066E7E0E076EBCEC01F007
:02124A00120090
:08124C00067EAAEC02F012007C
:101254000450000A08E10550000A05E1FF0E006E83
:101264007F0E016E58D00D6A096A086A0150001099
:10127400D8B4000C015005180A6E0ABE0D1E0B6A84
:1012840005AE05D0041E051E042AD8B4052A01AEF5
:1012940005D0001E011E002AD8B4012A01500510F1
:1012A4000A6E0ABE10D0D0EC04F00BB020D00DAE04
:1012B400000C001E011E002AD8B4012A081E091EB3
:1012C400082AD8B4092A000C05AE0DD001BE07D0F7
:1012D4000150096E0050086E016A006AE8D7016A7D
:1012E400006A002A000C011E001E0B2ADDD7082A02
:1012F400D8B4092A0450085CD8A4D9D70550095C8D
:10130400D8A4D5D7096A086A002AD8B4012A01AE3C
:08131400CED70000FF0C12000F
:10131C000450000A12E10550000A0FE10650000AC1
:10132C000CE10750000A09E1FF0E006EFF0E016E82
:10133C007F0E026EFF0E036EA8D0086A096A075072
:10134C00D8B439EF0AF00350D8B43EEF0AF002508B
:10135C0006180A6E028E068E0E6A02C008F001C0D4
:10136C000CF000C00DF004500D5E0550D8A0053CEB
:10137C000C5E0650D8A0063C085E086A0C6A0D6A22
:10138C00D8A0D0EF09F0D8900232013200320832E6
:10139C00010E0E6E0750035ED8A0DDEF09F07E0E35
:1013AC000E240326D8B043EF0AF0E3EF09F07E0ECB
:1013BC000E240326D8A048EF0AF0180E0B6E0D363B
:1013CC000C3608360036013602360E360450005EF6
:1013DC000550D8A0053C015E0650D8A0063C025E24
:1013EC0006340E120EA0FEEF09F00D8009EF0AF084
:1013FC00045000260550D8B0053C01260650D8B044
:10140C00062802260D900B2EE5EF09F02FEF0AF0BF
:10141C00D8900036013602360E360450005E055068
:10142C00D8A0053C015E0650D8A0063C025E0634EE
:10143C000E10010B0D26D8B00C2AD8B4082AD8A44B
:10144C002FEF0AF008320C320D32032AD8B443EFD6
:10145C000AF00AAE089E0850026E0C50016E0D5038
:10146C00006E4BEF0AF0010EB8EC01F04BEF0AF0F6
:10147C00020EAFEC00F04BEF0AF0040EA3EC00F000
:0C148C004BEF0AF0080EB6EC00F0120066
:10149800800E0101A219006E800E000A005CD8B00F
:1014A8006DD1A2510008016E01C0A2F1800E011891
:1014B800006E800E6E0A005CD8A0C0D0640E046E68
:1014C800A2C100F04CEC02F0120E0024056E000ED2
:1014D80000BEFF0E066E000E062205C000F006C014
:1014E80001F0000E06BEFF0E026E036E003600907D
:1014F80001360236033600360090013602360336CE
:10150800D10E0024F66E8A0E0120F76E000E02201E
:10151800F86E0900F5CFA3F10900F5CFA4F1090091
:10152800F5CFA5F10900F5CFA6F1640E046EA2C1AE
:1015380000F04CEC02F008C000F00A0E046E4CEC0F
:1015480002F0090E0024056E000E00BEFF0E066EA6
:10155800000E062205C000F006C001F0000E06BE0F
:10156800FF0E026E036E0036009001360236033617
:1015780000360090013602360336D10E0024F66E8E
:101588008A0E0120F76E000E0220F86E0900F5CFD2
:1015980000F00900F5CF01F00900F5CF02F00900CD
:1015A800F5CF03F0A3C104F0A4C105F0A5C106F06E
:1015B800A6C107F0BCEC01F000C0A3F101C0A4F182
:1015C80002C0A5F103C0A6F10A0E046EA2C100F084
:1015D8004CEC02F008C000F000C001F0000E00BEA4
:1015E800FF0E026E036E046E01360190023603365A
:1015F800043601360190023603360436D10E012432
:10160800F66E8A0E0220F76E000E0320F86E0900AF
:10161800F5CF00F00900F5CF01F00900F5CF02F091
:101628000900F5CF03F0A3C104F0A4C105F0A5C1DA
:1016380006F0A6C107F0BCEC01F007D2800E0A0A3A
:10164800006E800EA219005C71E20A0E046EA2C13F
:1016580000F04CEC02F0090E0024056E000E00BEEE
:10166800FF0E066E000E062205C000F006C001F04F
:10167800000E06BEFF0E026E036E003600900136A5
:101688000236033600360090013602360336D10E94
:101698000024F66E8A0E0120F76E000E0220F86E06
:1016A8000900F5CFA3F10900F5CFA4F10900F5CFA2
:1016B800A5F10900F5CFA6F10A0E046EA2C100F04B
:1016C8004CEC02F008C000F000C001F0000E00BEB3
:1016D800FF0E026E036E046E013601900236033669
:1016E800043601360190023603360436D10E012441
:1016F800F66E8A0E0220F76E000E0320F86E0900BF
:10170800F5CF00F00900F5CF01F00900F5CF02F0A0
:101718000900F5CF03F0A3C104F0A4C105F0A5C1E9
:1017280006F0A6C107F0BCEC01F08FD1A2C100F011
:10173800000EA2BFFF0E016E026E036E003600900F
:10174800013602360336003600900136023603367B
:10175800D10E0024F66E8A0E0120F76E000E0220CC
:10176800F86E0900F5CF00F00900F5CF01F0090087
:10177800F5CF02F00900F5CF03F067D1800EA2196A
:10178800006E800E6E0A005CD8A0C0D0640E046E95
:10179800A2C100F04CEC02F0120E0024056E000EFF
:1017A80000BEFF0E066E000E062205C000F006C041
:1017B80001F0000E06BEFF0E026E036E00360090AA
:1017C80001360236033600360090013602360336FB
:1017D800050E0024F66E8B0E0120F76E000E022017
:1017E800F86E0900F5CFA3F10900F5CFA4F10900BF
:1017F800F5CFA5F10900F5CFA6F1640E046EA2C1DC
:1018080000F04CEC02F008C000F00A0E046E4CEC3C
:1018180002F0090E0024056E000E00BEFF0E066ED3
:10182800000E062205C000F006C001F0000E06BE3C
:10183800FF0E026E036E0036009001360236033644
:1018480000360090013602360336050E0024F66E87
:101858008B0E0120F76E000E0220F86E0900F5CFFE
:1018680000F00900F5CF01F00900F5CF02F00900FA
:10187800F5CF03F0A3C104F0A4C105F0A5C106F09B
:10188800A6C107F0BCEC01F000C0A3F101C0A4F1AF
:1018980002C0A5F103C0A6F10A0E046EA2C100F0B1
:1018A8004CEC02F008C000F000C001F0000E00BED1
:1018B800FF0E026E036E046E013601900236033687
:1018C800043601360190023603360436050E01242B
:1018D800F66E8B0E0220F76E000E0320F86E0900DC
:1018E800F5CF00F00900F5CF01F00900F5CF02F0BF
:1018F8000900F5CF03F0A3C104F0A4C105F0A5C108
:1019080006F0A6C107F0BCEC01F09FD0800E0A0AD1
:10191800006E800EA219005C71E20A0E046EA2C16C
:1019280000F04CEC02F0090E0024056E000E00BE1B
:10193800FF0E066E000E062205C000F006C001F07C
:10194800000E06BEFF0E026E036E003600900136D2
:101958000236033600360090013602360336050E8D
:101968000024F66E8B0E0120F76E000E0220F86E32
:101978000900F5CFA3F10900F5CFA4F10900F5CFCF
:10198800A5F10900F5CFA6F10A0E046EA2C100F078
:101998004CEC02F008C000F000C001F0000E00BEE0
:1019A800FF0E026E036E046E013601900236033696
:1019B800043601360190023603360436050E01243A
:1019C800F66E8B0E0220F76E000E0320F86E0900EB
:1019D800F5CF00F00900F5CF01F00900F5CF02F0CE
:1019E8000900F5CF03F0A3C104F0A4C105F0A5C117
:1019F80006F0A6C107F0BCEC01F027D0A2C100F0A8
:101A0800000EA2BFFF0E016E026E036E003600903C
:101A180001360236033600360090013602360336A8
:101A2800050E0024F66E8B0E0120F76E000E0220C4
:101A3800F86E0900F5CF00F00900F5CF01F00900B4
:0C1A4800F5CF02F00900F5CF03F012000A
:101A54000050086E0150006E0250016E0350026E79
:101A6400036A0B6A0C6A9E0E036E0A6A020E0C6EFF
:061A7400C7EC00F01200B7
:101A7A0003500718D8A451EF0DF002500618D8A445
:101A8A0051EF0DF001500518D8A451EF0DF0005098
:0E1A9A000418D8B4D8841200D8941200120098
:101AA8000B6A0C6A0A6A086A0350D8B4DCEF0DF0B6
:101AB800028E9E0E035E03BE67EF0DF0D8B467EF8B
:101AC8000DF0CCEF0DF0036C080E035CD8A099EF75
:101AD8000DF0036E083600C008F001C000F002C027
:101AE80001F0026A080E035CD8A099EF0DF0036EAE
:101AF800083600C008F001C000F0016A080E035C57
:101B0800D8A099EF0DF0036E083600C008F0006AFF
:101B1800080E035CD8A099EF0DF0036E0836086A2A
:101B28000350D8A4D890A5EF0DF00350D8B4A5EF72
:101B38000DF0D8900232013200320832032E9DEFA8
:101B48000DF00BBC08A0B6EF0DF0D8A0B6EF0DF065
:101B5800082AD8B4002AD8B4012AD8B4022A02BE66
:101B6800E0EF0DF00AAEDCEF0DF0021E011E001EC4
:101B7800081E082AD8B4002AD8B4012AD8B4022AE0
:101B8800DCEF0DF0026A016A006A086ADCEF0DF00A
:101B98000B800BAEE6EF0DF0026A0AAEE6EF0DF031
:101BA800026E016E006E086E0A360232E6EF0DF024
:101BB800000E0C6AE7EF0DF0010E0C6EBBEC04F0A2
:101BC800E7EF0DF0FF0E0250036E0150026E005059
:081BD800016E0850006E1200BE
:0A1BE000A2C1A7F1C9EC04F0120045
:0C1BEA0072B201D0FDD7A2C173FF12003F
:101BF6000C6A0E6A0250D8A414EF0EF001C002F06F
:101C060000C001F0006A0E860250D8A414EF0EF050
:101C160001C002F0016A0E960E880250D8B426EF73
:101C26000EF00E50035ED8A4D8A02CEF0EF0D8907C
:101C360002BE32EF0EF0003601360236032E1BEFDF
:101C46000EF02CEF0EF0010E0C6EAFEC00F036EF3E
:101C56000EF0020E0C6EB6EC00F036EF0EF0040E2F
:081C66000C6EC3EC00F012004B
:101C6E00F250026EF29E0500FF6A0150FE6E0050A9
:081C7E00FD6E02BEF28E1200A1
:101C86006E0E01017A5DD8A0CAD0640E046E7AC1C8
:101C960000F09BEC02F0120E0024056E066A000EA0
:101CA600062205C000F006C001F0000E06BEFF0EBB
:101CB600026E036E00360090013602360336003699
:101CC60000900136023603366D0E0024F66E8B0E3A
:101CD6000120F76E000E0220F86E0900F5CF00F025
:101CE6000900F5CF01F00900F5CF02F00900F5CFA4
:101CF60003F0000E046E000E056E000E066E7E0EDC
:101D0600076EBCEC01F000C07BF101C07CF102C0A3
:101D16007DF103C07EF1640E046E7AC100F09BEC87
:101D260002F008C000F00A0E046E9BEC02F0090EE9
:101D36000024056E066A000E062205C000F006C0E5
:101D460001F0000E06BEFF0E026E036E0036009016
:101D56000136023603360036009001360236033667
:101D66006D0E0024F66E8B0E0120F76E000E02201B
:101D7600F86E0900F5CF00F00900F5CF01F0090073
:101D8600F5CF02F00900F5CF03F07BC104F07CC16A
:101D960005F07DC106F07EC107F0BCEC01F000C085
:101DA6007BF101C07CF102C07DF103C07EF10A0E19
:101DB600046E7AC100F09BEC02F008C000F000C08F
:101DC60001F0000E026E036E046E013601900236BB
:101DD60003360436013601900236033604366D0E9C
:101DE6000124F66E8B0E0220F76E000E0320F86EAD
:101DF6000900F5CF00F00900F5CF01F00900F5CF95
:101E060002F00900F5CF03F07BC104F07CC105F0B8
:101E16007DC106F07EC107F0BCEC01F0B1D07A516D
:101E26000A08D8B07ED00A0E046E7AC100F09BEC88
:101E360002F0090E0024056E066A000E062205C091
:101E460000F006C001F0000E06BEFF0E026E036E25
:101E56000036009001360236033600360090013611
:101E6600023603366D0E0024F66E8B0E0120F76ED9
:101E7600000E0220F86E0900F5CF00F00900F5CF3C
:101E860001F00900F5CF02F00900F5CF03F0000ECE
:101E9600046E000E056E000E066E7E0E076EBCEC1E
:101EA60001F000C07BF101C07CF102C07DF103C0EE
:101EB6007EF10A0E046E7AC100F09BEC02F008C0B7
:101EC60000F000C001F0000E026E036E046E0136D3
:101ED6000190023603360436013601900236033687
:101EE60004366D0E0124F66E8B0E0220F76E000E80
:101EF6000320F86E0900F5CF00F00900F5CF01F0D8
:101F06000900F5CF02F00900F5CF03F07BC104F01C
:101F16007CC105F07DC106F07EC107F0BCEC01F086
:101F26002FD07AC100F0000E016E026E036E0036ED
:101F3600009001360236033600360090013602362E
:101F460003366D0E0024F66E8B0E0120F76E000E22
:101F56000220F86E0900F5CF00F00900F5CF01F078
:101F66000900F5CF02F00900F5CF03F0000E046E6C
:101F7600000E056E000E066E7E0E076EBCEC01F0BE
:021F8600120047
:101F8800800E01017A19006E800E000A005CD8B03C
:101F98006DD17A510008016E01C07AF1800E0118E6
:101FA800006E800E6E0A005CD8A0C0D0640E046E6D
:101FB8007AC100F04CEC02F0120E0024056E000EFF
:101FC80000BEFF0E066E000E062205C000F006C019
:101FD80001F0000E06BEFF0E026E036E0036009082
:101FE80001360236033600360090013602360336D3
:101FF8006D0E0024F66E8B0E0120F76E000E022087
:10200800F86E0900F5CF7BF10900F5CF7CF10900E6
:10201800F5CF7DF10900F5CF7EF1640E046E7AC12B
:1020280000F04CEC02F008C000F00A0E046E4CEC14
:1020380002F0090E0024056E000E00BEFF0E066EAB
:10204800000E062205C000F006C001F0000E06BE14
:10205800FF0E026E036E003600900136023603361C
:10206800003600900136023603366D0E0024F66EF7
:102078008B0E0120F76E000E0220F86E0900F5CFD6
:1020880000F00900F5CF01F00900F5CF02F00900D2
:10209800F5CF03F07BC104F07CC105F07DC106F0EB
:1020A8007EC107F0BCEC01F000C07BF101C07CF1FF
:1020B80002C07DF103C07EF10A0E046E7AC100F001
:1020C8004CEC02F008C000F000C001F0000E00BEA9
:1020D800FF0E026E036E046E01360190023603365F
:1020E8000436013601900236033604366D0E01249B
:1020F800F66E8B0E0220F76E000E0320F86E0900B4
:10210800F5CF00F00900F5CF01F00900F5CF02F096
:102118000900F5CF03F07BC104F07CC105F07DC157
:1021280006F07EC107F0BCEC01F007D2800E0A0A67
:10213800006E800E7A19005C71E20A0E046E7AC194
:1021480000F04CEC02F0090E0024056E000E00BEF3
:10215800FF0E066E000E062205C000F006C001F054
:10216800000E06BEFF0E026E036E003600900136AA
:1021780002360336003600900136023603366D0EFD
:102188000024F66E8B0E0120F76E000E0220F86E0A
:102198000900F5CF7BF10900F5CF7CF10900F5CFF7
:1021A8007DF10900F5CF7EF10A0E046E7AC100F0C8
:1021B8004CEC02F008C000F000C001F0000E00BEB8
:1021C800FF0E026E036E046E01360190023603366E
:1021D8000436013601900236033604366D0E0124AA
:1021E800F66E8B0E0220F76E000E0320F86E0900C3
:1021F800F5CF00F00900F5CF01F00900F5CF02F0A6
:102208000900F5CF03F07BC104F07CC105F07DC166
:1022180006F07EC107F0BCEC01F08FD17AC100F066
:10222800000E7ABFFF0E016E026E036E003600903C
:102238000136023603360036009001360236033680
:102248006D0E0024F66E8B0E0120F76E000E022034
:10225800F86E0900F5CF00F00900F5CF01F009008C
:10226800F5CF02F00900F5CF03F067D1800E7A1997
:10227800006E800E6E0A005CD8A0C0D0640E046E9A
:102288007AC100F04CEC02F0120E0024056E000E2C
:1022980000BEFF0E066E000E062205C000F006C046
:1022A80001F0000E06BEFF0E026E036E00360090AF
:1022B8000136023603360036009001360236033600
:1022C800390E0024F66E8B0E0120F76E000E0220E8
:1022D800F86E0900F5CF7BF10900F5CF7CF1090014
:1022E800F5CF7DF10900F5CF7EF1640E046E7AC159
:1022F80000F04CEC02F008C000F00A0E046E4CEC42
:1023080002F0090E0024056E000E00BEFF0E066ED8
:10231800000E062205C000F006C001F0000E06BE41
:10232800FF0E026E036E0036009001360236033649
:1023380000360090013602360336390E0024F66E58
:102348008B0E0120F76E000E0220F86E0900F5CF03
:1023580000F00900F5CF01F00900F5CF02F00900FF
:10236800F5CF03F07BC104F07CC105F07DC106F018
:102378007EC107F0BCEC01F000C07BF101C07CF12C
:1023880002C07DF103C07EF10A0E046E7AC100F02E
:102398004CEC02F008C000F000C001F0000E00BED6
:1023A800FF0E026E036E046E01360190023603368C
:1023B800043601360190023603360436390E0124FC
:1023C800F66E8B0E0220F76E000E0320F86E0900E1
:1023D800F5CF00F00900F5CF01F00900F5CF02F0C4
:1023E8000900F5CF03F07BC104F07CC105F07DC185
:1023F80006F07EC107F0BCEC01F09FD0800E0A0AFF
:10240800006E800E7A19005C71E20A0E046E7AC1C1
:1024180000F04CEC02F0090E0024056E000E00BE20
:10242800FF0E066E000E062205C000F006C001F081
:10243800000E06BEFF0E026E036E003600900136D7
:102448000236033600360090013602360336390E5E
:102458000024F66E8B0E0120F76E000E0220F86E37
:102468000900F5CF7BF10900F5CF7CF10900F5CF24
:102478007DF10900F5CF7EF10A0E046E7AC100F0F5
:102488004CEC02F008C000F000C001F0000E00BEE5
:10249800FF0E026E036E046E01360190023603369B
:1024A800043601360190023603360436390E01240B
:1024B800F66E8B0E0220F76E000E0320F86E0900F0
:1024C800F5CF00F00900F5CF01F00900F5CF02F0D3
:1024D8000900F5CF03F07BC104F07CC105F07DC194
:1024E80006F07EC107F0BCEC01F027D07AC100F0FD
:1024F800000E7ABFFF0E016E026E036E003600906A
:1025080001360236033600360090013602360336AD
:10251800390E0024F66E8B0E0120F76E000E022095
:10252800F86E0900F5CF00F00900F5CF01F00900B9
:0C253800F5CF02F00900F5CF03F012000F
:1025440001017A51200A09E07A510D0804E3090EC9
:102554007A5D01E302D0006A02D0010E006E12001F
:10256400220E0C6E086A096A0A6A0B6A0C06D8B451
:102574001FD0D8900B320A320932083203320232A9
:1025840001320032D8A0F2D70C06D8B409D00450D6
:1025940008260550092206500A2207500B22EAD7C2
:1025A400045008260550092206500A2207500B221F
:0225B400120013
:1025B60001019A6B9B6B8E6B8F6B7CC100F07DC1AA
:1025C60001F07EC102F0010E7C27000E7D237E23E2
:1025D60000C0F6FF01C0F7FF02C0F8FF0900F5CF03
:1025E60000F000C08BF10052D8B4EBEF22F08B5113
:1025F600250A0BE07AC1E1FF7BC1E2FF8BC1E6FF52
:102606007A4B7B2B9A4B9B2BD8D78C6B8D6B8E6B17
:102616008F6B23D08E87010E7C27000E7D237E23B1
:1026260059D08E81010E7C27000E7D237E2352D049
:102636008E83010E7C27000E7D237E234BD08F8751
:10264600010E7C27000E7D237E2344D08E85010E4D
:102656007C27000E7D237E233DD07CC1F6FF7DC105
:10266600F7FF7EC1F8FF0900F5CF01F001502D0AF2
:10267600D1E07CC1F6FF7DC1F7FF7EC1F8FF0900FE
:10268600F5CF01F00150200ACCE07CC1F6FF7DC1F8
:10269600F7FF7EC1F8FF0900F5CF01F001502B0AC4
:1026A600C7E07CC1F6FF7DC1F7FF7EC1F8FF0900D8
:1026B600F5CF01F00150230AC2E07CC1F6FF7DC1CF
:1026C600F7FF7EC1F8FF0900F5CF01F00150300A8F
:1026D600BDE001D09ED78EA301D08E918EA701D0EA
:1026E6008E957CC1F6FF7DC1F7FF7EC1F8FF09001C
:1026F600F5CF00F0000E016E00C0A2F199EC07F0D4
:10270600005236E08C6B8D6B8CC100F08DC101F0F0
:102716000A0E046E000E056E72EC06F07CC1F6FF22
:102726007DC1F7FF7EC1F8FF0900F5CF02F0025028
:1027360000248C6F000E01208D6F300E8C5F000E12
:102746008D5B010E7C27000E7D237E237CC1F6FF68
:102756007DC1F7FF7EC1F8FF0900F5CF00F0000E3E
:10276600016E00C0A2F199EC07F00052CDE133D022
:102776007CC1F6FF7DC1F7FF7EC1F8FF0900F5CFEA
:1027860001F001502A0A27E17FC1E9FF80C1EAFF73
:10279600EECF00F0EECF01F000C0E9FF01C0EAFF86
:1027A600EECF8CF1EECF8DF17FC1E9FF80C1EAFF5C
:1027B600020EEE24006E000EEE20016E7FC1E1FFD8
:1027C60080C1E2FF00C0E6FF01C0E6FF010E7C27E4
:1027D600000E7D237E237CC1F6FF7DC1F7FF7EC1FF
:1027E600F8FF0900F5CF01F001502E0A70E1010E45
:1027F6007C27000E7D237E237CC1F6FF7DC1F7FF7B
:102806007EC1F8FF0900F5CF01F001502A0A28E140
:102816007FC1E9FF80C1EAFFEECF00F0EECF01F005
:1028260000C0E9FF01C0EAFFEECF89F1EECF8AF1E1
:102836007FC1E9FF80C1EAFF020EEE24006E000EA2
:10284600EE20016E7FC1E1FF80C1E2FF00C0E6FF1E
:1028560001C0E6FF010E7C27000E7D237E2336D0C5
:10286600896B8A6B7CC1F6FF7DC1F7FF7EC1F8FFDD
:102876000900F5CF00F0000E016E00C0A2F199EC40
:1028860007F0005223E089C100F08AC101F00A0E68
:10289600046E000E056E72EC06F07CC1F6FF7DC17B
:1028A600F7FF7EC1F8FF0900F5CF02F002500024C1
:1028B600896F000E01208A6F300E895F000E8A5BD9
:1028C600010E7C27000E7D237E23CCD703D0896B97
:1028D6008A6B8F897CC100F07DC101F07EC102F058
:1028E600010E7C27000E7D237E2300C0F6FF01C06B
:1028F600F7FF02C0F8FF0900F5CF8BF1F9D09AC1B6
:1029060000F09BC101F0EFEF22F08E89E3D78F85AF
:102916002ED18E8B8F812BD18F8329D18E8D27D16E
:1029260026D18E8B8E8F23D17FC1E9FF80C1EAFF2E
:10293600EECF00F0EECF01F000C0E9FF01C0EAFFE4
:10294600EECF96F1EECF97F17FC1E9FF80C1EAFFA6
:10295600020EEE24006E000EEE20016E7FC1E1FF36
:1029660080C1E2FF00C0E6FF01C0E6FF000E971936
:1029760002E1000E961904E1240E966F000E976F81
:10298600986B996B98519625E96E99519721EA6E45
:10299600EE520BE0010E9825006E000E9921016E95
:1029A60000C098F101C099F1EDD789518A110AE06A
:1029B60099518A5D02E19851895D04E289C198F1D5
:1029C6008AC199F18D51995D02E18C51985D05E2BC
:1029D60098518C5F99518D5B02D08C6B8D6B8EB745
:1029E60016D08CC100F08DC101F0010E8C5F000E77
:1029F6008D5B005001100BE07AC1E1FF7BC1E2FF65
:102A0600200EE66E7A4B7B2B9A4B9B2BEAD798C10E
:102A160002F099C103F0010E985D006E000E9959FF
:102A2600016E00C098F101C099F10250031019E03F
:102A360096C1E9FF97C1EAFF7AC1E1FF7BC1E2FFD8
:102A4600EECFE6FF7A4B7B2B010E9625006E000E2D
:102A56009721016E00C096F101C097F19A4B9B2B0E
:102A6600D6D78EA716D08CC100F08DC101F0010E0D
:102A76008C5F000E8D5B005001100BE07AC1E1FF08
:102A86007BC1E2FF200EE66E7A4B7B2B9A4B9B2B8B
:102A9600EAD793D57FC1E9FF80C1EAFFEECF00F008
:102AA600EECF01F000C0E9FF01C0EAFFEECF8BF1E7
:102AB6007FC1E9FF80C1EAFF020EEE24006E000E20
:102AC600EE20016E7FC1E1FF80C1E2FF00C0E6FF9C
:102AD60001C0E6FF8B0E966F010E976F010E986F81
:102AE600000E996F62D7C00E8E13000E8F133FD063
:102AF6008B51000AD8B403D78B516C0AD8B405D7CA
:102B06008B514C0AD8B401D78B51660AD8B4FFD67C
:102B16008B51450AD8B4FDD68B51650AD8B4FAD67E
:102B26008B51670AD8B4F8D68B516F0AD8B4F6D64B
:102B36008B51640AD8B4F4D68B51690AD8B4F0D64E
:102B46008B51700AD8B4EDD68B51580AD8B4E9D651
:102B56008B51780AD8B4E6D68B51730AD8B4E4D62A
:102B66008B51630A97E08B51750ABDE0B3D7000E0F
:102B76008E15006E8F51070B016E00500110D8B4F0
:102B860092EF1EF08FA904D0060E896F000E8A6F91
:102B96007FC1E9FF80C1EAFFEECF00F0EECF01F082
:102BA60000C0E9FF01C0EAFFEECF90F1EECF91F150
:102BB600EECF92F1EECF93F17FC1E9FF80C1EAFF3C
:102BC600040EEE24006E000EEE20016E7FC1E1FFC2
:102BD60080C1E2FF00C0E6FF01C0E6FF046A056AA5
:102BE600066A076A90C100F091C101F092C102F035
:102BF60093C103F09AEC06F0010ED8B0000E006EF9
:102C0600005205E0927F030E8E13000E8F13946B15
:102C1600956B90C100F091C101F092C102F093C191
:102C260003F0046A056A066A076A3DEC0DF0000EB9
:102C3600D8A4010E006E0052D8B48AD093C100F019
:102C4600016A026A036AFF0E0016000E01167E0E66
:102C5600005E000E015A00C094F101C095F1010E0C
:102C6600005E000E015A00C094F101C095F1030EFA
:102C7600046E000E056E72EC06F000C094F101C001
:102C860095F10A0E046E000E056E2AEC09F000C0DE
:102C960094F101C095F1800E0118026E800E025C5F
:102CA60002E1000E005C05E2010E0101945F000ED8
:102CB600955B010194510008A26F4CEC0AF090C19B
:102CC60004F091C105F092C106F093C107F0BCEC87
:102CD60001F000C096F101C097F102C098F103C05F
:102CE60099F1000E046E000E056E000E066E7F0E44
:102CF600076E96C100F097C101F098C102F099C124
:102D060003F09AEC06F0010ED8B0000E006E0052E9
:102D160005E0010E945F000E955B1AD0000E046E5E
:102D2600000E056E200E066E820E076E96C100F02E
:102D360097C101F098C102F099C103F09AEC06F030
:102D4600000ED8B0010E006E005202E0944B952B97
:102D5600800E006E800E9519005C02E19451000809
:102D660003E3010E8B6F02D094C18BF18FB118D0A3
:102D76008FA315D0800E9519006E7F0E005C02E1C0
:102D8600FC0E945D0BE3800E9519006E800E8A1979
:102D9600005C02E18951945D01E201D001D0F1D3DA
:102DA60089518A1106E08FA304D0010E895F000EB7
:102DB6008A5B000E006E8A51005C02E189510808A8
:102DC60003E2080E8B6F02D089C18BF190C100F02F
:102DD60091C101F092C102F093C103F0046A056A41
:102DE600066A076A3DEC0DF0000ED8A4010E006ECF
:102DF6000052D8B44BD194C1A2F14CEC0AF000C0F9
:102E060004F001C005F002C006F003C007F090C14F
:102E160000F091C101F092C102F093C103F08EEC73
:102E260009F000C090F101C091F102C092F103C017
:102E360093F101018B510008A26F4CEC0AF000C01F
:102E460004F001C005F002C006F003C007F090C10F
:102E560000F091C101F092C102F093C103F08EEC33
:102E660009F000C09CF101C09DF102C09EF103C0B3
:102E76009FF19CC190F19DC191F19EC192F19FC1BC
:102E860093F19CC100F09DC101F09EC102F09FC16B
:102E960003F054EC0DF02AEC0DF000C004F001C074
:102EA60005F002C006F003C007F09CC100F09DC10A
:102EB60001F09EC102F09FC103F026EC09F0000E5E
:102EC600046E000E056E000E066E7E0E076E9AEC00
:102ED60006F0000ED8B0010E006E00521AE090C146
:102EE60000F091C101F092C102F093C103F0000E0F
:102EF600046E000E056E000E066E7E0E076EAAECC0
:102F060002F000C090F101C091F102C092F103C03D
:102F160093F190C100F091C101F092C102F093C10A
:102F260003F054EC0DF001018B51010F096E0A6A92
:102F3600000E0A2209C004F00AC005F0000E0ABEFF
:102F4600FF0E066E076E0436049005360636073603
:102F560004360490053606360736290E0424F66E26
:102F66008C0E0520F76E000E0620F86E0900F5CFD0
:102F760005F00900F5CF06F00900F5CF07F00900C6
:102F8600F5CF08F00850035C08E10750025C05E144
:102F96000650015C02E10550005C1EE3010190C190
:102FA60000F091C101F092C102F093C103F0CD0E81
:102FB600046ECC0E056E4C0E066E7B0E076EBCECD8
:102FC60001F000C090F101C091F102C092F103C07E
:102FD60093F1944B952B5AD090C100F091C101F01A
:102FE60092C102F093C103F054EC0DF08BC104F0D2
:102FF600000E056E066E076E04360490053606361C
:10300600073604360490053606360736290E04249C
:10301600F66E8C0E0520F76E000E0620F86E09007F
:10302600F5CF05F00900F5CF06F00900F5CF07F05A
:103036000900F5CF08F00850035C08E10750025C70
:1030460005E10650015C02E10550005C1FE201014A
:1030560090C100F091C101F092C102F093C103F05A
:10306600000E046E000E056E200E066E820E076EB2
:10307600BCEC01F000C090F101C091F102C092F1E8
:1030860003C093F1010E945F000E955B01018FA3BF
:1030960093D08FB791D0800E000A006E800E8A19E9
:1030A600005C02E189510A0804E20A0E896F000EEB
:1030B6008A6F90C100F091C101F092C102F093C1F4
:1030C60003F054EC0DF000C096F101C097F102C078
:1030D60098F103C099F1965197119811991142E010
:1030E6000A0E046E000E056E066E076E96C100F09F
:1030F60097C101F098C102F099C103F0FCEC04F00D
:1031060008C000F009C001F00AC002F00BC003F0CD
:10311600000E046E031808E10450021805E104507D
:10312600011802E10050000A1DE1010E895F000E40
:103136008A5B0A0E046E000E056E066E076E96C159
:1031460000F097C101F098C102F099C103F0FCECC0
:1031560004F000C096F101C097F102C098F103C0D7
:1031660099F1B9D7800E8A19006E800E005C02E1D3
:103176008B51895D21E289518B5DA26F4CEC0AF07F
:1031860000C004F001C005F002C006F003C007F05D
:1031960090C100F091C101F092C102F093C103F019
:1031A6008EEC09F000C090F101C091F102C092F1DD
:1031B60003C093F189C18BF1050E01018925006ECB
:1031C600000E8A21016E00508C5F01508D5B895183
:1031D6008A1103E18FB701D004D0010E8C5F000E77
:1031E6008D5B030E8E15006E8FC101F0000E011669
:1031F6000050011004E0010E8C5F000E8D5B8EA561
:1032060039D08EA312D08EA103D02D0E816F02D09D
:103216002B0E816F7AC1E1FF7BC1E2FF81C1E6FF20
:103226007A4B7B2B9A4B9B2B0CD08EA10AD07AC162
:10323600E1FF7BC1E2FF200EE66E7A4B7B2B9A4BB9
:103246009B2B800E006E800E8D19005C02E18C5166
:1032560000080FE27AC1E1FF7BC1E2FF300EE66EA5
:103266007A4B7B2B9A4B9B2B010E8C5F000E8D5B52
:10327600E8D73AD08EB718D0800E006E800E8D1922
:10328600005C02E18C5100080FE27AC1E1FF7BC1CC
:10329600E2FF200EE66E7A4B7B2B9A4B9B2B010EA0
:1032A6008C5F000E8D5BE8D78EA312D08EA103D063
:1032B6002D0E826F02D02B0E826F7AC1E1FF7BC189
:1032C600E2FF82C1E6FF7A4B7B2B9A4B9B2B0CD0FD
:1032D6008EA10AD07AC1E1FF7BC1E2FF200EE66E25
:1032E6007A4B7B2B9A4B9B2B90C100F091C101F03E
:1032F60092C102F093C103F054EC0DF000C096F1B8
:1033060001C097F102C098F103C099F18BC100F09A
:10331600000E016E026E036E003600900136023614
:10332600033600360090013602360336290E002495
:10333600F66E8C0E0120F76E000E0220F86E090064
:10334600F5CF04F00900F5CF05F00900F5CF06F03A
:103356000900F5CF07F096C100F097C101F098C1BA
:1033660002F099C103F0FCEC04F0300E00267AC19D
:10337600E1FF7BC1E2FF00C0E6FF7A4B7B2B9A4B55
:103386009B2B89518A1103E18FB701D06FD07AC187
:10339600E1FF7BC1E2FF2E0EE66E7A4B7B2B9A4B4A
:1033A6009B2B8B51895F000E8A5B8B534DE08B07FD
:1033B6008BC100F0000E016E026E036E00360090A7
:1033C60001360236033600360090013602360336E1
:1033D600290E0024F66E8C0E0120F76E000E0220D8
:1033E600F86E0900F5CF04F00900F5CF05F00900E5
:1033F600F5CF06F00900F5CF07F096C100F097C1AA
:1034060001F098C102F099C103F0FCEC04F00A0E39
:10341600046E000E056E066E076EFCEC04F008C026
:1034260000F009C001F00AC002F00BC003F0300E34
:1034360000267AC1E1FF7BC1E2FF00C0E6FF7A4BBE
:103446007B2B9A4B9B2BB1D789518A110FE07AC1FE
:10345600E1FF7BC1E2FF300EE66E7A4B7B2B9A4B87
:103466009B2B010E895F000E8A5BEED78EAB0BD0CD
:103476007AC1E1FF7BC1E2FF450EE66E7A4B7B2BFC
:103486009A4B9B2B0AD07AC1E1FF7BC1E2FF650E06
:10349600E66E7A4B7B2B9A4B9B2B800E9519006E12
:1034A600800E005C02E1000E945D11E2945100086A
:1034B600946F9551000E95577AC1E1FF7BC1E2FFEB
:1034C6002D0EE66E7A4B7B2B9A4B9B2B0AD07AC13C
:1034D600E1FF7BC1E2FF2B0EE66E7A4B7B2B9A4B0C
:1034E6009B2B0A0E046E000E056E94C100F095C16A
:1034F60001F02AEC09F0300E00267AC1E1FF7BC10B
:10350600E2FF00C0E6FF01017A4B7B2B9A4B9B2B17
:103516000A0E046E000E056E94C100F095C101F00E
:103526002AEC09F008C000F009C001F0300E0026B0
:103536007AC1E1FF7BC1E2FF00C0E6FF01017A4BE1
:103546007B2B9A4B9B2B8EA71AD0800E006E800E7B
:103556008D19005C02E18C51000811E27AC1E1FF8D
:103566007BC1E2FF200EE66E7A4B7B2B9A4B9B2BA0
:10357600010E8C5F000E8D5B8C518D11EFE1E0EF3B
:1035860012F08FA3F3D0800E9519006E800E005CAA
:1035960002E1000E945D0AE2010E945D006E000EDB
:1035A6009559016E0050895F01508A5B90C100F009
:1035B60091C101F092C102F093C103F054EC0DF0F9
:1035C60000C096F101C097F102C098F103C099F1CD
:1035D600010E8B6F8B510A0A34E08BC100F0000E8E
:1035E600016E026E036E0036009001360236033617
:1035F60000360090013602360336290E0024F66E98
:103606008C0E0120F76E000E0220F86E0900F5CF31
:1036160001F00900F5CF02F00900F5CF03F009002B
:10362600F5CF04F00450995D08E10350985D05E17B
:103636000250975D02E10150965D01E202D08B2BAC
:10364600C9D78B51895DA06F000E8A59A16FA0C1A1
:1036560089F1A1C18AF196C100F097C101F098C124
:1036660002F099C103F02AEC0DF000C004F001C08D
:1036760005F002C006F003C007F090C100F091C14A
:1036860001F092C102F093C103F026EC09F000C0EC
:103696009CF101C09DF102C09EF103C09FF1A0C143
:1036A600A2F14CEC0AF09CC104F09DC105F09EC14C
:1036B60006F09FC107F0BCEC01F0000E046E000E90
:1036C600056E000E066E7E0E076EAAEC02F054EC36
:1036D6000DF000C096F101C097F102C098F103C049
:1036E60099F189518A1142E00A0E046E000E056EA8
:1036F600066E076E96C100F097C101F098C102F000
:1037060099C103F0FCEC04F008C000F009C001F018
:103716000AC002F00BC003F0000E046E031808E1A5
:103726000450021805E10450011802E10050000A95
:103736001DE10A0E046E000E056E066E076E96C13A
:1037460000F097C101F098C102F099C103F0FCECBA
:1037560004F000C096F101C097F102C098F103C0D1
:1037660099F1010E895F000E8A5BBBD7800E006E51
:10377600800E8A19005C02E189510C0816E389C1A2
:10378600A2F1A5EC07F090C104F091C105F092C139
:1037960006F093C107F0AAEC02F000C090F101C058
:1037A60091F102C092F103C093F190C100F091C172
:1037B60001F092C102F093C103F0046A056A066A39
:1037C600076A3DEC0DF0000ED8A4010E006E005203
:1037D600D8B477D090C100F091C101F092C102F047
:1037E60093C103F054EC0DF0000E046E031808E1CB
:1037F6000450021805E10450011802E10050000AC5
:1038060060E1800E006E800E9519005C02E1945115
:10381600010857E294C1A2F14CEC0AF000C004F092
:1038260001C005F002C006F003C007F090C100F029
:1038360091C101F092C102F093C103F08EEC09F040
:103846005F0E046E700E056E090E066E810E076E13
:103856009AEC06F0010ED8B0000E006E005206E09B
:10386600090E0101945F000E955B05D00101080E5B
:10387600945F000E955B94C1A2F14CEC0AF000C077
:1038860004F001C005F002C006F003C007F090C1C5
:1038960000F091C101F092C102F093C103F08EECE9
:1038A60009F054EC0DF000C096F101C097F102C08A
:1038B60098F103C099F10101906B916B926B936B38
:1038C60038D090C100F091C101F092C102F093C1CD
:1038D60003F054EC0DF000C096F101C097F102C060
:1038E60098F103C099F196C100F097C101F098C113
:1038F60002F099C103F02AEC0DF000C004F001C0FB
:1039060005F002C006F003C007F090C100F091C1B7
:1039160001F092C102F093C103F026EC09F000C059
:1039260090F101C091F102C092F103C093F1946B42
:10393600956B010E8B6F8B510A0A34E08BC100F038
:10394600000E016E026E036E0036009001360236DE
:10395600033600360090013602360336290E00245F
:10396600F66E8C0E0120F76E000E0220F86E09002E
:10397600F5CF01F00900F5CF02F00900F5CF03F00D
:103986000900F5CF04F00450995D08E10350985DF5
:1039960005E10250975D02E10150965D01E202D019
:1039A6008B2BC9D78B518925006E000E8A21016E9B
:1039B600945100269551012200508C5F01508D5B79
:1039C6008FB704D089518A1101E104D0010E8C5FB2
:1039D600000E8D5B030E8E15006E8FC101F0000E7A
:1039E60001160050011004E0010E8C5F000E8D5B85
:1039F6008EA539D08EA312D08EA103D02D0E836F43
:103A060002D02B0E836F7AC1E1FF7BC1E2FF83C137
:103A1600E6FF7A4B7B2B9A4B9B2B0CD08EA10AD0C0
:103A26007AC1E1FF7BC1E2FF200EE66E7A4B7B2B6B
:103A36009A4B9B2B800E006E800E8D19005C02E166
:103A46008C5100080FE27AC1E1FF7BC1E2FF300E24
:103A5600E66E7A4B7B2B9A4B9B2B010E8C5F000EEE
:103A66008D5BE8D73AD08EB718D0800E006E800EE8
:103A76008D19005C02E18C5100080FE27AC1E1FF6A
:103A86007BC1E2FF200EE66E7A4B7B2B9A4B9B2B7B
:103A9600010E8C5F000E8D5BE8D78EA312D08EA12F
:103AA60003D02D0E846F02D02B0E846F7AC1E1FFF6
:103AB6007BC1E2FF84C1E6FF7A4B7B2B9A4B9B2BA3
:103AC6000CD08EA10AD07AC1E1FF7BC1E2FF200EA5
:103AD600E66E7A4B7B2B9A4B9B2B8BC100F08B07A8
:103AE60000524CE08BC100F0000E016E026E036EB8
:103AF6000036009001360236033600360090013655
:103B060002360336290E0024F66E8C0E0120F76E5F
:103B1600000E0220F86E0900F5CF04F00900F5CF7B
:103B260005F00900F5CF06F00900F5CF07F096C1BC
:103B360000F097C101F098C102F099C103F0FCECC6
:103B460004F00A0E046E000E056E066E076EFCEC9F
:103B560004F008C000F009C001F00AC002F00BC072
:103B660003F0300E00267AC1E1FF7BC1E2FF00C000
:103B7600E6FF7A4B7B2B9A4B9B2BAFD7800E006EC2
:103B8600800E9519005C02E1945100080FE27AC19B
:103B9600E1FF7BC1E2FF300EE66E7A4B7B2B9A4B40
:103BA6009B2B010E945F000E955BE8D7800E000AF2
:103BB600006E800E8A19005C02E18951080803E252
:103BC600080E8B6F02D089C18BF18B51895F000E75
:103BD6008A5B8B5303E18FB701D00AD07AC1E1FF2C
:103BE6007BC1E2FF2E0EE66E7A4B7B2B9A4B9B2B0C
:103BF6008BC1A2F14CEC0AF090C104F091C105F022
:103C060092C106F093C107F0BCEC01F001EC07F09D
:103C160000C096F101C097F102C098F103C099F176
:103C26008B534DE08B078BC100F0000E016E026EC8
:103C3600036E0036009001360236033600360090D9
:103C4600013602360336290E0024F66E8C0E01204C
:103C5600F76E000E0220F86E0900F5CF04F0090099
:103C6600F5CF05F00900F5CF06F00900F5CF07F00E
:103C760096C100F097C101F098C102F099C103F016
:103C8600FCEC04F00A0E046E000E056E066E076E5E
:103C9600FCEC04F008C000F009C001F00AC002F014
:103CA6000BC003F0300E00267AC1E1FF7BC1E2FFB4
:103CB60000C0E6FF7A4B7B2B9A4B9B2BB1D78951E1
:103CC6008A110FE07AC1E1FF7BC1E2FF300EE66E9A
:103CD6007A4B7B2B9A4B9B2B010E895F000E8A5BDE
:103CE600EED78EA71AD0800E006E800E8D19005C5E
:103CF60002E18C51000811E27AC1E1FF7BC1E2FFCB
:103D0600200EE66E7A4B7B2B9A4B9B2B010E8C5F1B
:103D1600000E8D5B8C518D11EFE1E0EF12F0C00EBD
:103D26008E15016E8FC102F0000E0216000E0218EB
:103D360002E1000E0118D8A480D08EA927D07FC139
:103D4600E9FF80C1EAFFEECF00F0EECF01F000C040
:103D5600E9FF01C0EAFFEECF96F1EECF97F1EECF85
:103D660098F1EECF99F17FC1E9FF80C1EAFF040E19
:103D7600EE24006E000EEE20016E7FC1E1FF80C1D1
:103D8600E2FF00C0E6FF01C0E6FF2FD07FC1E9FFDA
:103D960080C1EAFFEECF00F0EECF01F000C0E9FFF0
:103DA60001C0EAFFEECF00F0EECF01F0000E01BE3B
:103DB600FF0E026E036E00C096F101C097F102C0BD
:103DC60098F103C099F17FC1E9FF80C1EAFF020EB5
:103DD600EE24006E000EEE20016E7FC1E1FF80C171
:103DE600E2FF00C0E6FF01C0E6FF800E9919006EF3
:103DF600800E005C08E1000E985D05E1000E975DFF
:103E060002E1000E965D18E2030E8E13000E8F136C
:103E1600006A016A026A036A9651005E9751015A66
:103E26009851025A9951035A00C096F101C097F170
:103E360002C098F103C099F14ED08EA927D07FC158
:103E4600E9FF80C1EAFFEECF00F0EECF01F000C03F
:103E5600E9FF01C0EAFFEECF96F1EECF97F1EECF84
:103E660098F1EECF99F17FC1E9FF80C1EAFF040E18
:103E7600EE24006E000EEE20016E7FC1E1FF80C1D0
:103E8600E2FF00C0E6FF01C0E6FF25D07FC1E9FFE3
:103E960080C1EAFFEECF00F0EECF01F000C0E9FFEF
:103EA60001C0EAFFEECF96F1EECF97F1000E986FC4
:103EB600996F7FC1E9FF80C1EAFF020EEE24006E12
:103EC600000EEE20016E7FC1E1FF80C1E2FF00C05F
:103ED600E6FF01C0E6FF000E8A1902E1000E89190D
:103EE6000FE1000E006E991908E10050981905E1DE
:103EF6000050971902E19651000A02E1894B8A2B7C
:103F0600C00E8E15006E00C005F0AED0010E8B6F90
:103F16008B510A0A34E08BC100F0000E016E026E6E
:103F2600036E0036009001360236033600360090E6
:103F3600013602360336290E0024F66E8C0E012059
:103F4600F76E000E0220F86E0900F5CF01F00900A9
:103F5600F5CF02F00900F5CF03F00900F5CF04F024
:103F66000450995D08E10350985D05E10250975DA4
:103F760002E10150965D01E202D08B2BC9D782D0B7
:103F8600010E8B6F8B51080A34E08BC100F0000ED6
:103F9600016E026E036E003600900136023603365D
:103FA60000360090013602360336890E0024F66E7E
:103FB6008D0E0120F76E000E0220F86E0900F5CF77
:103FC60001F00900F5CF02F00900F5CF03F0090072
:103FD600F5CF04F00450995D08E10350985D05E1C2
:103FE6000250975D02E10150965D01E202D08B2BF3
:103FF600C9D748D0010E8B6F8B510C0A34E08BC1A8
:1040060000F0000E016E026E036E0036009001365F
:104016000236033600360090013602360336D10EDC
:104026000024F66E8B0E0120F76E000E0220F86E4D
:104036000900F5CF01F00900F5CF02F00900F5CF30
:1040460003F00900F5CF04F00450995D08E1035030
:10405600985D05E10250975D02E10150965D01E22F
:1040660002D08B2BC9D70ED00550000AD8B44ED734
:104076000550C00AD8B44AD70550800A81E00550D9
:10408600400AB8E0800E006E800E8A19005C02E1DC
:1040960089518B5D03E289C18BF10DD0800E8A199F
:1040A600006E800E005C02E18B51895D04E28BC1DB
:1040B60089F1000E8A6F8C518D110EE0030E8E155C
:1040C600006E8FC101F0000E01160050011004E0D1
:1040D600010E8C5F000E8D5B800E8A19006E800EBD
:1040E6008D19005C02E18C51895D05E289518C5F76
:1040F6008A518D5B02D08C6B8D6BC40E8E15016E52
:104106008F51080B026E0250080A02E1400E011898
:1041160008E18C518D1104E0010E8C5F000E8D5B61
:104126001CD0C00E8E15016E8F51080B026E025008
:10413600080A02E1800E011810E1800E006E800E62
:104146008D19005C02E18C51020805E2020E8C5FBB
:10415600000E8D5B02D08C6B8D6B8EA55DD08EA311
:1041660012D08EA103D02D0E856F02D02B0E856F37
:104176007AC1E1FF7BC1E2FF85C1E6FF7A4B7B2B6B
:104186009A4B9B2B34D08EA10BD07AC1E1FF7BC119
:10419600E2FF200EE66E7A4B7B2B9A4B9B2B27D0A9
:1041A600C00E8E15016E8F51080B026E0250080A62
:1041B60002E1800E01181BE17AC1E1FF7BC1E2FF3B
:1041C600300EE66E7A4B7B2B9A4B9B2B8EAB03D035
:1041D600580E866F02D0780E866F7AC1E1FF7BC1DA
:1041E600E2FF86C1E6FF7A4B7B2B9A4B9B2B8C51C9
:1041F6008D1111E07AC1E1FF7BC1E2FF300EE66E60
:104206007A4B7B2B9A4B9B2B010E8C5F000E8D5BA2
:104216008C518D11EFE174D08C518D1113E08EB756
:1042260011D07AC1E1FF7BC1E2FF200EE66E7A4B28
:104236007B2B9A4B9B2B010E8C5F000E8D5B8C515A
:104246008D11EFE18EA312D08EA103D02D0E876FB4
:1042560002D02B0E876F7AC1E1FF7BC1E2FF87C1D7
:10426600E6FF7A4B7B2B9A4B9B2B0CD08EA10AD068
:104276007AC1E1FF7BC1E2FF200EE66E7A4B7B2B13
:104286009A4B9B2BC00E8E15016E8F51080B026E3A
:104296000250080A02E1400E01180BE17AC1E1FF63
:1042A6007BC1E2FF300EE66E7A4B7B2B9A4B9B2B43
:1042B60027D0C00E8E15016E8F51080B026E02506C
:1042C600080A02E1800E01181BE17AC1E1FF7BC1F9
:1042D600E2FF300EE66E7A4B7B2B9A4B9B2B8EAB16
:1042E60003D0580E886F02D0780E886F7AC1E1FF2E
:1042F6007BC1E2FF88C1E6FF7A4B7B2B9A4B9B2B57
:10430600800E006E800E8A19005C02E189518B5D79
:104316000BE27AC1E1FF7BC1E2FF300EE66E7A4B1B
:104326007B2B9A4B9B2BECD789C100F08AC101F0FD
:10433600010E895F000E8A5B00500110D8B42AD1A5
:10434600C00E8E15006E00C09CF10AD189C100F026
:104356008AC101F0000E8ABFFF0E026E036E0036A0
:1043660000900136023603360036009001360236DA
:104376000336290E0024F66E8C0E0120F76E000E11
:104386000220F86E0900F5CF04F00900F5CF05F01C
:104396000900F5CF06F00900F5CF07F096C100F049
:1043A60097C101F098C102F099C103F0FCEC04F04A
:1043B6000A0E046E000E056E066E076EFCEC04F027
:1043C60008C000F009C001F00AC002F00BC003F0FB
:1043D600300E00248B6FD3D08EAB45D089C100F050
:1043E6008AC101F0000E8ABFFF0E026E036E003610
:1043F600009001360236033600360090013602364A
:104406000336890E0024F66E8D0E0120F76E000E1F
:104416000220F86E0900F5CF04F00900F5CF05F08B
:104426000900F5CF06F00900F5CF07F096C100F0B8
:1044360097C101F098C102F099C103F0FCEC04F0B9
:104446000F0E0016000E011602160316AF0E0024FC
:10445600F66E8E0E0120F76E000E0220F86E090031
:10446600F5CF8BF144D089C100F08AC101F0000E6E
:104476008ABFFF0E026E036E0036009001360236CA
:10448600033600360090013602360336890E0024C4
:10449600F66E8D0E0120F76E000E0220F86E0900F2
:1044A600F5CF04F00900F5CF05F00900F5CF06F0C9
:1044B6000900F5CF07F096C100F097C101F098C149
:1044C60002F099C103F0FCEC04F00F0E0016000E8A
:1044D6000116021603168D0E0024F66E8E0E0120AE
:1044E600F76E000E0220F86E0900F5CF8BF147D06B
:1044F60089C100F08AC101F0000E8ABFFF0E026E6C
:10450600036E003600900136023603360036009000
:10451600013602360336D10E0024F66E8B0E0120CC
:10452600F76E000E0220F86E0900F5CF04F00900C0
:10453600F5CF05F00900F5CF06F00900F5CF07F035
:1045460096C100F097C101F098C102F099C103F03D
:10455600FCEC04F0070E00148B6F300E8B270FD087
:104566009C51000AD8B4F2D69C51C00AD8B4EED6F3
:104576009C51800AD8B430D79C51400AB9E07AC120
:10458600E1FF7BC1E2FF8BC1E6FF7A4B7B2B9A4BA7
:104596009B2BCAD68EA71AD0800E006E800E8D1960
:1045A600005C02E18C51000811E27AC1E1FF7BC197
:1045B600E2FF200EE66E7A4B7B2B9A4B9B2B010E6D
:1045C6008C5F000E8D5B8C518D11EFE1E0EF12F0E8
:0A45D6009AC100F09BC101F0120031
:1045E0000050086E0150006E0250016E0350026EC2
:1045F000036A0B6A0C6A9E0E036E0A6A02AE0DEF26
:1046000023F0081E001E011E021E082AD8B4002A2C
:10461000D8B4012AD8B4022A0A8E020E0C6EC7EC56
:0446200000F0120094
:10462400C7B409D01F0EC514016E0150000A03E17E
:0A463400010E006E01D0006A1200B2
:10463E0053C100F0016A026A036AFF0E0016000EF3
:10464E00011600C058F101C059F17F0E005C026ED8
:10465E00000E0158036E02C058F103C059F1800ECE
:10466E000318006E800E005C02E1000E025C22E276
:10467E00046A056A066A076A50C100F051C101F06A
:10468E0052C102F053C103F09AEC06F0010ED8B0FD
:10469E00000E006E005209E0000E006E000E016E5C
:1046AE00800E026E7F0E036E5DD0006A016A026A92
:1046BE00036A58D0000E006E01015951005C02E1F0
:1046CE005851180809E250C100F051C101F052C111
:1046DE0002F053C103F046D050C100F051C101F0B9
:1046EE0052C102F053C103F001EC07F072DF00C0BB
:1046FE0054F101C055F102C056F103C057F100C08C
:10470E0004F001C005F002C006F003C007F050C16E
:10471E0000F051C101F052C102F053C103F09AEC06
:10472E0006F0010ED8B0000E006E005213E0000E1F
:10473E00046E000E056E000E066E7F0E076E54C1DF
:10474E0000F055C101F056C102F057C103F026EC3E
:10475E0009F008D054C100F055C101F056C102F065
:06476E0057C103F0120028
:104774000101566B576B000E575D02E10A0E565D40
:104784000BE256515425E16E57515521E26E200E2D
:10479400E66E564B572BEFD756515425E16E5751C1
:1047A4005521E26EE66A010E565F000E575B5651C4
:1047B4005425586F57515521596F0A0E046E000E37
:1047C400056E066E076E50C100F051C101F052C172
:1047D40002F053C103F0FCEC04F008C000F009C07F
:1047E40001F00AC002F00BC003F0300E002658C1DD
:1047F400E1FF59C1E2FF00C0E6FF0A0E046E000E9D
:10480400056E066E076E50C100F051C101F052C131
:1048140002F053C103F0FCEC04F000C050F101C0FD
:1048240051F102C052F103C053F1000E046E03189B
:1048340008E10450021805E10450011802E1005097
:10484400000A01E105D0010E565F000E575BAFD799
:02485400120050
:104856000101726B736B666B676B010154C100F0EB
:1048660055C101F056C102F0010E5427000E552322
:10487600562300C0F6FF01C0F7FF02C0F8FF09008B
:10488600F5CF00F000C063F10052D8B4C7EF34F0A2
:104896006351250A0DE052C1E1FF53C1E2FF63C136
:1048A600E6FF50C100F051C101F037EC0EF0D5D74C
:1048B6000101646B656B666B676B24D001016687CB
:1048C600010E5427000E5523562359D06681010E3A
:1048D6005427000E5523562352D06683010E5427C3
:1048E600000E552356234BD06787010E5427000E22
:1048F6005523562344D06685010E5427000E5523B2
:1049060056233DD054C1F6FF55C1F7FF56C1F8FFF7
:104916000900F5CF01F001502D0AD0E054C1F6FF91
:1049260055C1F7FF56C1F8FF0900F5CF01F0015058
:10493600200ACCE054C1F6FF55C1F7FF56C1F8FF77
:104946000900F5CF01F001502B0AC7E054C1F6FF6C
:1049560055C1F7FF56C1F8FF0900F5CF01F0015028
:10496600230AC2E054C1F6FF55C1F7FF56C1F8FF4E
:104976000900F5CF01F00150300ABDE001D09DD706
:1049860066A301D0669166A701D0669554C1F6FF6D
:1049960055C1F7FF56C1F8FF0900F5CF00F0000E2C
:1049A600016E00C0A2F199EC07F0005236E0646B8C
:1049B600656B64C100F065C101F00A0E046E000E5D
:1049C600056E72EC06F054C1F6FF55C1F7FF56C1ED
:1049D600F8FF0900F5CF02F002500024646F000EC4
:1049E6000120656F300E645F000E655B010E542773
:1049F600000E5523562354C1F6FF55C1F7FF56C185
:104A0600F8FF0900F5CF00F0000E016E00C0A2F11C
:104A160099EC07F00052CDE133D054C1F6FF55C1F1
:104A2600F7FF56C1F8FF0900F5CF01F001502A0A39
:104A360027E157C1E9FF58C1EAFFEECF00F0EECFFC
:104A460001F000C0E9FF01C0EAFFEECF64F1EECF4E
:104A560065F157C1E9FF58C1EAFF020EEE24006E68
:104A6600000EEE20016E57C1E1FF58C1E2FF00C003
:104A7600E6FF01C0E6FF010E5427000E552356231C
:104A860054C1F6FF55C1F7FF56C1F8FF0900F5CF2F
:104A960001F001502E0A70E1010E5427000E552335
:104AA600562354C1F6FF55C1F7FF56C1F8FF09005A
:104AB600F5CF01F001502A0A28E157C1E9FF58C194
:104AC600EAFFEECF00F0EECF01F000C0E9FF01C033
:104AD600EAFFEECF61F1EECF62F157C1E9FF58C1AF
:104AE600EAFF020EEE24006E000EEE20016E57C1A4
:104AF600E1FF58C1E2FF00C0E6FF01C0E6FF010E7C
:104B06005427000E5523562336D0616B626B54C171
:104B1600F6FF55C1F7FF56C1F8FF0900F5CF00F0C3
:104B2600000E016E00C0A2F199EC07F0005223E0DE
:104B360061C100F062C101F00A0E046E000E056E3E
:104B460072EC06F054C1F6FF55C1F7FF56C1F8FFE7
:104B56000900F5CF02F002500024616F000E01201B
:104B6600626F300E615F000E625B010E5427000E0D
:104B760055235623CCD703D0616B626B678954C12A
:104B860000F055C101F056C102F0010E5427000E87
:104B96005523562300C0F6FF01C0F7FF02C0F8FFF9
:104BA6000900F5CF63F104D172C100F073C101F0C1
:104BB600CBEF34F06689E3D7678539D1668B678199
:104BC60036D1678334D1668D32D131D1668B668F0B
:104BD6002ED157C1E9FF58C1EAFFEECF00F0EECF64
:104BE60001F000C0E9FF01C0EAFFEECF6EF1EECFA3
:104BF6006FF157C1E9FF58C1EAFF020EEE24006EBD
:104C0600000EEE20016E57C1E1FF58C1E2FF00C061
:104C1600E6FF01C0E6FF000E6F1902E1000E6E19F5
:104C260004E11D0E6E6F000E6F6F706B716B70512D
:104C36006E25E96E71516F21EA6EEE520BE0010EA0
:104C46007025006E000E7121016E00C070F101C06A
:104C560071F1EDD7615162110AE07151625D02E1B5
:104C66007051615D04E261C170F162C171F165511B
:104C7600715D02E16451705D05E27051645F7151CE
:104C8600655B02D0646B656B66B719D0010164C1C0
:104C960000F065C101F0010E645F000E655B005017
:104CA60001100DE052C1E1FF53C1E2FF200EE66E96
:104CB60050C100F051C101F037EC0EF0E7D770C1DA
:104CC60002F071C103F0010E0101705D006E000E6D
:104CD6007159016E00C070F101C071F102500310EC
:104CE6001CE052C1E1FF53C1E2FF6EC1E9FF6FC193
:104CF600EAFFEECFE6FF50C100F051C101F037ECFC
:104D06000EF0010E01016E25006E000E6F21016E80
:104D160000C06EF101C06FF1D2D766A719D00101AC
:104D260064C100F065C101F0010E645F000E655BB1
:104D3600005001100DE052C1E1FF53C1E2FF200E09
:104D4600E66E50C100F051C101F037EC0EF0E7D726
:104D560084D557C1E9FF58C1EAFFEECF00F0EECF88
:104D660001F000C0E9FF01C0EAFFEECF63F157C1D1
:104D7600E9FF58C1EAFF020EEE24006E000EEE2097
:104D8600016E57C1E1FF58C1E2FF00C0E6FF01C056
:104D9600E6FF630E01016E6F010E6F6F010E706FFD
:104DA600000E716F57D7C00E6613000E67133FD003
:104DB6006351000AD8B4F8D663516C0AD8B4FAD64F
:104DC60063514C0AD8B4F6D66351660AD8B4F4D601
:104DD6006351450AD8B4F2D66351650AD8B4EFD602
:104DE6006351670AD8B4EDD663516F0AD8B4EBD6CF
:104DF6006351640AD8B4E9D66351690AD8B4E5D6D2
:104E06006351700AD8B4E2D66351580AD8B4DED6D4
:104E16006351780AD8B4DBD66351730AD8B4D9D6AD
:104E26006351630A96E06351750ABDE0B2D7000E7E
:104E36006615006E6751070B016E00500110D8B45D
:104E460044EF30F067A904D0060E616F000E626F62
:104E560057C1E9FF58C1EAFFEECF00F0EECF01F0EF
:104E660000C0E9FF01C0EAFFEECF68F1EECF69F1BD
:104E7600EECF6AF1EECF6BF157C1E9FF58C1EAFFF9
:104E8600040EEE24006E000EEE20016E57C1E1FF07
:104E960058C1E2FF00C0E6FF01C0E6FF046A056AEA
:104EA600066A076A68C100F069C101F06AC102F0CA
:104EB6006BC103F09AEC06F0010ED8B0000E006E3E
:104EC600005205E06A7F030E6613000E67136C6BD3
:104ED6006D6B68C100F069C101F06AC102F06BC177
:104EE60003F0046A056A066A076A3DEC0DF0000ED7
:104EF600D8A4010E006E0052D8B48AD06BC100F05F
:104F0600016A026A036AFF0E0016000E01167E0E83
:104F1600005E000E015A00C06CF101C06DF1010E79
:104F2600005E000E015A00C06CF101C06DF1030E67
:104F3600046E000E056E72EC06F000C06CF101C046
:104F46006DF10A0E046E000E056E2AEC09F000C023
:104F56006CF101C06DF1800E0118026E800E025CCC
:104F660002E1000E005C05E2010E01016C5F000E1D
:104F76006D5B01016C5100087A6FC4EC0FF068C1DB
:104F860004F069C105F06AC106F06BC107F0BCEC1C
:104F960001F000C06EF101C06FF102C070F103C0F4
:104FA60071F1000E046E000E056E000E066E7F0E89
:104FB600076E6EC100F06FC101F070C102F071C1E1
:104FC60003F09AEC06F0010ED8B0000E006E005207
:104FD60005E0010E6C5F000E6D5B1AD0000E046ECC
:104FE600000E056E200E066E820E076E6EC100F074
:104FF6006FC101F070C102F071C103F09AEC06F0C6
:10500600000ED8B0010E006E005202E06C4B6D2B04
:10501600800E006E800E6D19005C02E16C51000876
:1050260003E3010E636F02D06CC163F167B119D05F
:1050360067A315D0800E6D19006E7F0E005C02E12D
:10504600FC0E6C5D0BE3800E6D19006E800E62190E
:10505600005C02E161516C5D01E201D002D052EFC9
:105066002CF06151621106E067A304D0010E615F66
:10507600000E625B000E006E6251005C02E161513F
:10508600080803E2080E636F02D061C163F168C1CC
:1050960000F069C101F06AC102F06BC103F0046A55
:1050A600056A066A076A3DEC0DF0000ED8A4010EEB
:1050B600006E0052D8B44BD16CC17AF1C4EC0FF03B
:1050C60000C004F001C005F002C006F003C007F0FE
:1050D60068C100F069C101F06AC102F06BC103F05A
:1050E6008EEC09F000C068F101C069F102C06AF1F6
:1050F60003C06BF10101635100087A6FC4EC0FF035
:1051060000C004F001C005F002C006F003C007F0BD
:1051160068C100F069C101F06AC102F06BC103F019
:105126008EEC09F000C074F101C075F102C076F191
:1051360003C077F174C168F175C169F176C16AF18E
:1051460077C16BF174C100F075C101F076C102F050
:1051560077C103F054EC0DF02AEC0DF000C004F01A
:1051660001C005F002C006F003C007F074C100F0EC
:1051760075C101F076C102F077C103F026EC09F0A3
:10518600000E046E000E056E000E066E7E0E076E95
:105196009AEC06F0000ED8B0010E006E00521AE02E
:1051A60068C100F069C101F06AC102F06BC103F089
:1051B600000E046E000E056E000E066E7E0E076E65
:1051C600AAEC02F000C068F101C069F102C06AF100
:1051D60003C06BF168C100F069C101F06AC102F059
:1051E6006BC103F054EC0DF001016351010F096E20
:1051F6000A6A000E0A2209C004F00AC005F0000E71
:105206000ABEFF0E066E076E043604900536063695
:10521600073604360490053606360736010E042492
:10522600F66E8C0E0520F76E000E0620F86E09004D
:10523600F5CF05F00900F5CF06F00900F5CF07F028
:105246000900F5CF08F00850035C08E10750025C3E
:1052560005E10650015C02E10550005C1EE3010118
:1052660068C100F069C101F06AC102F06BC103F0C8
:10527600CD0E046ECC0E056E4C0E066E7B0E076EC2
:10528600BCEC01F000C068F101C069F102C06AF12E
:1052960003C06BF16C4B6D2B5AD068C100F069C12D
:1052A60001F06AC102F06BC103F054EC0DF063C16A
:1052B60004F0000E056E066E076E04360490053681
:1052C6000636073604360490053606360736010ECE
:1052D6000424F66E8C0E0520F76E000E0620F86E7E
:1052E6000900F5CF05F00900F5CF06F00900F5CF66
:1052F60007F00900F5CF08F00850035C08E10750F5
:10530600025C05E10650015C02E10550005C1FE20B
:10531600010168C100F069C101F06AC102F06BC108
:1053260003F0000E046E000E056E200E066E820E51
:10533600076EBCEC01F000C068F101C069F102C063
:105346006AF103C06BF1010E6C5F000E6D5B01012B
:1053560067A393D067B791D0800E000A006E800EC7
:105366006219005C02E161510A0804E20A0E616FEB
:10537600000E626F68C100F069C101F06AC102F0F7
:105386006BC103F054EC0DF000C06EF101C06FF17B
:1053960002C070F103C071F16E516F11701171117D
:1053A60042E00A0E046E000E056E066E076E6EC1B2
:1053B60000F06FC101F070C102F071C103F0FCECA6
:1053C60004F008C000F009C001F00AC002F00BC0EA
:1053D60003F0000E046E031808E10450021805E1FC
:1053E6000450011802E10050000A1DE1010E615F40
:1053F600000E625B0A0E046E000E056E066E076EE8
:105406006EC100F06FC101F070C102F071C103F00E
:10541600FCEC04F000C06EF101C06FF102C070F147
:1054260003C071F1B9D7800E6219006E800E005C60
:1054360002E16351615D21E26151635D7A6FC4EC03
:105446000FF000C004F001C005F002C006F003C072
:1054560007F068C100F069C101F06AC102F06BC1D2
:1054660003F08EEC09F000C068F101C069F102C0DA
:105476006AF103C06BF161C163F1050E010161259B
:10548600006E000E6221016E0050645F0150655B84
:105496006151621103E167B701D004D0010E645F68
:1054A600000E655B030E6615006E67C101F0000E07
:1054B60001160050011004E0010E645F000E655BEA
:1054C60066A542D066A314D066A103D02D0E596FEF
:1054D60002D02B0E596F52C1E1FF53C1E2FF59C1F1
:1054E600E6FF50C100F051C101F037EC0EF00FD0CD
:1054F600010166A10CD052C1E1FF53C1E2FF200EAB
:10550600E66E50C100F051C101F037EC0EF0800E8E
:10551600006E800E01016519005C02E1645100080D
:1055260012E252C1E1FF53C1E2FF300EE66E50C1F6
:1055360000F051C101F037EC0EF0010E0101645F7D
:10554600000E655BE4D742D066B71BD0800E006EB6
:10555600800E6519005C02E16451000812E252C136
:10556600E1FF53C1E2FF200EE66E50C100F051C1CB
:1055760001F037EC0EF0010E0101645F000E655B71
:10558600E5D766A314D066A103D02D0E5A6F02D0BC
:105596002B0E5A6F52C1E1FF53C1E2FF5AC1E6FF1B
:1055A60050C100F051C101F037EC0EF00FD00101EF
:1055B60066A10CD052C1E1FF53C1E2FF200EE66E98
:1055C60050C100F051C101F037EC0EF068C100F097
:1055D60069C101F06AC102F06BC103F054EC0DF031
:1055E60000C06EF101C06FF102C070F103C071F12D
:1055F60063C100F0000E016E026E036E003600906D
:10560600013602360336003600900136023603367E
:10561600010E0024F66E8C0E0120F76E000E02209D
:10562600F86E0900F5CF04F00900F5CF05F0090082
:10563600F5CF06F00900F5CF07F06EC100F06FC197
:1056460001F070C102F071C103F0FCEC04F0300E01
:10565600002652C1E1FF53C1E2FF00C0E6FF50C180
:1056660000F051C101F037EC0EF0010161516211F9
:1056760003E167B701D079D052C1E1FF53C1E2FF20
:105686002E0EE66E50C100F051C101F037EC0EF05F
:1056960001016351615F000E625B010163534FE0DC
:1056A600630763C100F0000E016E026E036E0036E2
:1056B6000090013602360336003600900136023677
:1056C6000336010E0024F66E8C0E0120F76E000ED6
:1056D6000220F86E0900F5CF04F00900F5CF05F0B9
:1056E6000900F5CF06F00900F5CF07F06EC100F00E
:1056F6006FC101F070C102F071C103F0FCEC04F05F
:105706000A0E046E000E056E066E076EFCEC04F0C3
:1057160008C000F009C001F00AC002F00BC003F097
:10572600300E002652C1E1FF53C1E2FF00C0E6FF82
:1057360050C100F051C101F037EC0EF0AED70101B7
:105746006151621112E052C1E1FF53C1E2FF300E16
:10575600E66E50C100F051C101F037EC0EF0010EBB
:105766000101615F000E625BEAD766AB0DD052C1E4
:10577600E1FF53C1E2FF450EE66E50C100F051C194
:1057860001F037EC0EF00CD052C1E1FF53C1E2FF3D
:10579600650EE66E50C100F051C101F037EC0EF017
:1057A600800E01016D19006E800E005C02E1000E94
:1057B6006C5D13E26C5100086C6F6D51000E6D57F5
:1057C60052C1E1FF53C1E2FF2D0EE66E50C100F05B
:1057D60051C101F037EC0EF00CD052C1E1FF53C1BC
:1057E600E2FF2B0EE66E50C100F051C101F037EC1E
:1057F6000EF00A0E046E000E056E6CC100F06DC14F
:1058060001F02AEC09F0300E002652C1E1FF53C127
:10581600E2FF00C0E6FF50C100F051C101F037ECD5
:105826000EF00A0E046E000E056E6CC100F06DC11E
:1058360001F02AEC09F008C000F009C001F0300EB2
:10584600002652C1E1FF53C1E2FF00C0E6FF50C18E
:1058560000F051C101F037EC0EF0010166A71DD032
:10586600800E006E800E6519005C02E1645100082E
:1058760014E252C1E1FF53C1E2FF200EE66E50C1B1
:1058860000F051C101F037EC0EF0010E0101645F2A
:10589600000E655B64516511ECE130EF24F067A3FF
:1058A600F3D0800E6D19006E800E005C02E1000ED2
:1058B6006C5D0AE2010E6C5D006E000E6D59016EA4
:1058C6000050615F0150625B68C100F069C101F080
:1058D6006AC102F06BC103F054EC0DF000C06EF12A
:1058E60001C06FF102C070F103C071F1010E636F68
:1058F60063510A0A34E063C100F0000E016E026EC5
:10590600036E0036009001360236033600360090EC
:10591600013602360336010E0024F66E8C0E012087
:10592600F76E000E0220F86E0900F5CF01F00900AF
:10593600F5CF02F00900F5CF03F00900F5CF04F02A
:105946000450715D08E10350705D05E102506F5D22
:1059560002E101506E5D01E202D0632BC9D76351AB
:10596600615D786F000E6259796F78C161F179C116
:1059760062F16EC100F06FC101F070C102F071C139
:1059860003F02AEC0DF000C004F001C005F002C0DF
:1059960006F003C007F068C100F069C101F06AC1F2
:1059A60002F06BC103F026EC09F000C074F101C0EF
:1059B60075F102C076F103C077F178C17AF1C4ECD3
:1059C6000FF074C104F075C105F076C106F077C119
:1059D60007F0BCEC01F0000E046E000E056E000E22
:1059E600066E7E0E076EAAEC02F054EC0DF000C0B7
:1059F6006EF101C06FF102C070F103C071F1615127
:105A0600621142E00A0E046E000E056E066E076E07
:105A16006EC100F06FC101F070C102F071C103F0F8
:105A2600FCEC04F008C000F009C001F00AC002F066
:105A36000BC003F0000E046E031808E104500218B0
:105A460005E10450011802E10050000A1DE10A0EAA
:105A5600046E000E056E066E076E6EC100F06FC115
:105A660001F070C102F071C103F0FCEC04F000C05B
:105A76006EF101C06FF102C070F103C071F1010E49
:105A8600615F000E625BBBD7800E006E800E6219EE
:105A9600005C02E161510C0816E361C17AF143EC46
:105AA6000EF068C104F069C105F06AC106F06BC169
:105AB60007F0AAEC02F000C068F101C069F102C06B
:105AC6006AF103C06BF168C100F069C101F06AC1F7
:105AD60002F06BC103F0046A056A066A076A3DECC8
:105AE6000DF0000ED8A4010E006E0052D8B477D087
:105AF60068C100F069C101F06AC102F06BC103F030
:105B060054EC0DF0000E046E031808E10450021860
:105B160005E10450011802E10050000A60E1800E20
:105B2600006E800E6D19005C02E16C51010857E2AF
:105B36006CC17AF1C4EC0FF000C004F001C005F0AE
:105B460002C006F003C007F068C100F069C101F0A9
:105B56006AC102F06BC103F08EEC09F05F0E046EB1
:105B6600700E056E090E066E810E076E9AEC06F033
:105B7600010ED8B0000E006E005206E0090E0101BB
:105B86006C5F000E6D5B05D00101080E6C5F000EA8
:105B96006D5B6CC17AF1C4EC0FF000C004F001C07B
:105BA60005F002C006F003C007F068C100F069C145
:105BB60001F06AC102F06BC103F08EEC09F054ECFF
:105BC6000DF000C06EF101C06FF102C070F103C0AC
:105BD60071F10101686B696B6A6B6B6B38D068C1D8
:105BE60000F069C101F06AC102F06BC103F054EC28
:105BF6000DF000C06EF101C06FF102C070F103C07C
:105C060071F16EC100F06FC101F070C102F071C197
:105C160003F02AEC0DF000C004F001C005F002C04C
:105C260006F003C007F068C100F069C101F06AC15F
:105C360002F06BC103F026EC09F000C068F101C068
:105C460069F102C06AF103C06BF16C6B6D6B010EFA
:105C5600636F63510A0A34E063C100F0000E016EFF
:105C6600026E036E003600900136023603360036A9
:105C76000090013602360336010E0024F66E8C0EB5
:105C86000120F76E000E0220F86E0900F5CF01F034
:105C96000900F5CF02F00900F5CF03F00900F5CFB2
:105CA60004F00450715D08E10350705D05E1025097
:105CB6006F5D02E101506E5D01E202D0632BC9D730
:105CC60063516125006E000E6221016E6C51002643
:105CD6006D5101220050645F0150655B67B704D0C7
:105CE6006151621101E104D0010E645F000E655B33
:105CF600030E6615006E67C101F0000E0116005016
:105D0600011004E0010E645F000E655B66A542D0DB
:105D160066A314D066A103D02D0E5B6F02D02B0EA6
:105D26005B6F52C1E1FF53C1E2FF5BC1E6FF50C1A9
:105D360000F051C101F037EC0EF00FD0010166A161
:105D46000CD052C1E1FF53C1E2FF200EE66E50C1F6
:105D560000F051C101F037EC0EF0800E006E800E9F
:105D660001016519005C02E16451000812E252C1AA
:105D7600E1FF53C1E2FF300EE66E50C100F051C1A3
:105D860001F037EC0EF0010E0101645F000E655B59
:105D9600E4D742D066B71BD0800E006E800E651920
:105DA600005C02E16451000812E252C1E1FF53C1F6
:105DB600E2FF200EE66E50C100F051C101F037EC53
:105DC6000EF0010E0101645F000E655BE5D766A368
:105DD60014D066A103D02D0E5C6F02D02B0E5C6F23
:105DE60052C1E1FF53C1E2FF5CC1E6FF50C100F0C2
:105DF60051C101F037EC0EF00FD0010166A10CD0B5
:105E060052C1E1FF53C1E2FF200EE66E50C100F021
:105E160051C101F037EC0EF063C100F001016307D8
:105E260000524EE063C100F0000E016E026E036E7A
:105E360000360090013602360336003600900136F1
:105E460002360336010E0024F66E8C0E0120F76E24
:105E5600000E0220F86E0900F5CF04F00900F5CF18
:105E660005F00900F5CF06F00900F5CF07F06EC181
:105E760000F06FC101F070C102F071C103F0FCECDB
:105E860004F00A0E046E000E056E066E076EFCEC3C
:105E960004F008C000F009C001F00AC002F00BC00F
:105EA60003F0300E002652C1E1FF53C1E2FF00C0ED
:105EB600E6FF50C100F051C101F037EC0EF0ACD74F
:105EC600800E006E800E01016D19005C02E16C51BE
:105ED600000812E252C1E1FF53C1E2FF300EE66E46
:105EE60050C100F051C101F037EC0EF0010E010176
:105EF6006C5F000E6D5BE4D7800E000A006E800EAC
:105F06006219005C02E16151080803E2080E636F42
:105F160002D061C163F16351615F000E625B63533E
:105F260003E167B701D00CD052C1E1FF53C1E2FFD4
:105F36002E0EE66E50C100F051C101F037EC0EF0A6
:105F460063C17AF1C4EC0FF068C104F069C105F0D1
:105F56006AC106F06BC107F0BCEC01F001EC07F07A
:105F660000C06EF101C06FF102C070F103C071F1A3
:105F7600010163534FE0630763C100F0000E016E39
:105F8600026E036E00360090013602360336003686
:105F96000090013602360336010E0024F66E8C0E92
:105FA6000120F76E000E0220F86E0900F5CF04F00E
:105FB6000900F5CF05F00900F5CF06F00900F5CF89
:105FC60007F06EC100F06FC101F070C102F071C13F
:105FD60003F0FCEC04F00A0E046E000E056E066E6D
:105FE600076EFCEC04F008C000F009C001F00AC01E
:105FF60002F00BC003F0300E002652C1E1FF53C180
:10600600E2FF00C0E6FF50C100F051C101F037ECDD
:106016000EF0AED701016151621112E052C1E1FFEB
:1060260053C1E2FF300EE66E50C100F051C101F0DF
:1060360037EC0EF0010E0101615F000E625BEAD7DC
:1060460066A71DD0800E006E800E6519005C02E109
:106056006451000814E252C1E1FF53C1E2FF200E71
:10606600E66E50C100F051C101F037EC0EF0010EA2
:106076000101645F000E655B64516511ECE130EF70
:1060860024F0C00E6615016E67C102F0000E0216FE
:10609600000E021802E1000E0118D8A480D066A9ED
:1060A60027D057C1E9FF58C1EAFFEECF00F0EECF87
:1060B60001F000C0E9FF01C0EAFFEECF6EF1EECFBE
:1060C6006FF1EECF70F1EECF71F157C1E9FF58C114
:1060D600EAFF040EEE24006E000EEE20016E57C19C
:1060E600E1FF58C1E2FF00C0E6FF01C0E6FF2FD086
:1060F60057C1E9FF58C1EAFFEECF00F0EECF01F03D
:1061060000C0E9FF01C0EAFFEECF00F0EECF01F0DC
:10611600000E01BEFF0E026E036E00C06EF101C0DE
:106126006FF102C070F103C071F157C1E9FF58C1A8
:10613600EAFF020EEE24006E000EEE20016E57C13D
:10614600E1FF58C1E2FF00C0E6FF01C0E6FF800E96
:106156007119006E800E005C08E1000E705D05E1AD
:10616600000E6F5D02E1000E6E5D18E2030E66130F
:10617600000E6713006A016A026A036A6E51005EC6
:106186006F51015A7051025A7151035A00C06EF193
:1061960001C06FF102C070F103C071F14ED066A963
:1061A60027D057C1E9FF58C1EAFFEECF00F0EECF86
:1061B60001F000C0E9FF01C0EAFFEECF6EF1EECFBD
:1061C6006FF1EECF70F1EECF71F157C1E9FF58C113
:1061D600EAFF040EEE24006E000EEE20016E57C19B
:1061E600E1FF58C1E2FF00C0E6FF01C0E6FF25D08F
:1061F60057C1E9FF58C1EAFFEECF00F0EECF01F03C
:1062060000C0E9FF01C0EAFFEECF6EF1EECF6FF1FD
:10621600000E706F716F57C1E9FF58C1EAFF020E99
:10622600EE24006E000EEE20016E57C1E1FF58C14C
:10623600E2FF00C0E6FF01C0E6FF000E621902E1C0
:10624600000E61190FE1000E006E711908E1005091
:10625600701905E100506F1902E16E51000A02E162
:10626600614B622BC00E6615006E00C005F0AED005
:10627600010E636F63510A0A34E063C100F0000E39
:10628600016E026E036E003600900136023603364A
:1062960000360090013602360336010E0024F66EF3
:1062A6008C0E0120F76E000E0220F86E0900F5CF65
:1062B60001F00900F5CF02F00900F5CF03F009005F
:1062C600F5CF04F00450715D08E10350705D05E1FF
:1062D60002506F5D02E101506E5D01E202D0632B58
:1062E600C9D782D0010E636F6351080A34E063C1D7
:1062F60000F0000E016E026E036E0036009001364D
:106306000236033600360090013602360336290E71
:106316000024F66E8D0E0120F76E000E0220F86E38
:106326000900F5CF01F00900F5CF02F00900F5CF1D
:1063360003F00900F5CF04F00450715D08E1035045
:10634600705D05E102506F5D02E101506E5D01E294
:1063560002D0632BC9D748D0010E636F63510C0A74
:1063660034E063C100F0000E016E026E036E00366B
:1063760000900136023603360036009001360236AA
:106386000336A10E0024F66E8B0E0120F76E000E6A
:106396000220F86E0900F5CF01F00900F5CF02F0F2
:1063A6000900F5CF03F00900F5CF04F00450715D44
:1063B60008E10350705D05E102506F5D02E1015096
:1063C6006E5D01E202D0632BC9D70ED00550000ADC
:1063D600D8B44ED70550C00AD8B44AD70550800A5B
:1063E60081E00550400AB8E0800E006E800E62190A
:1063F600005C02E16151635D03E261C163F10DD0AE
:10640600800E6219006E800E005C02E16351615DD0
:1064160004E263C161F1000E626F645165110EE022
:10642600030E6615006E67C101F0000E01160050DE
:10643600011004E0010E645F000E655B800E6219B8
:10644600006E800E6519005C02E16451615D05E233
:106456006151645F6251655B02D0646B656BC40E0B
:106466006615016E6751080B026E0250080A02E1BA
:10647600400E011808E16451651104E0010E645FE5
:10648600000E655B1CD0C00E6615016E6751080BC9
:10649600026E0250080A02E1800E011810E1800E19
:1064A600006E800E6519005C02E16451020805E287
:1064B600020E645F000E655B02D0646B656B66A5B9
:1064C6006CD066A314D066A103D02D0E5D6F02D0EA
:1064D6002B0E5D6F52C1E1FF53C1E2FF5DC1E6FFC6
:1064E60050C100F051C101F037EC0EF03DD0010172
:1064F60066A10DD052C1E1FF53C1E2FF200EE66E48
:1065060050C100F051C101F037EC0EF02DD0C00E95
:1065160001016615016E6751080B026E0250080AEA
:1065260002E1800E011820E152C1E1FF53C1E2FFF2
:10653600300EE66E50C100F051C101F037EC0EF09E
:10654600010166AB03D0580E5E6F02D0780E5E6F07
:1065560052C1E1FF53C1E2FF5EC1E6FF50C100F048
:1065660051C101F037EC0EF001016451651114E0E0
:1065760052C1E1FF53C1E2FF300EE66E50C100F09A
:1065860051C101F037EC0EF0010E0101645F000EFF
:10659600655B64516511ECE185D06451651116E0C7
:1065A60066B714D052C1E1FF53C1E2FF200EE66E7A
:1065B60050C100F051C101F037EC0EF0010E01019F
:1065C600645F000E655B64516511ECE166A314D04F
:1065D60066A103D02D0E5F6F02D02B0E5F6F52C1E6
:1065E600E1FF53C1E2FF5FC1E6FF50C100F051C1B8
:1065F60001F037EC0EF00FD0010166A10CD052C1AC
:10660600E1FF53C1E2FF200EE66E50C100F051C11A
:1066160001F037EC0EF0C00E01016615016E6751F0
:10662600080B026E0250080A02E1400E01180DE145
:1066360052C1E1FF53C1E2FF300EE66E50C100F0D9
:1066460051C101F037EC0EF02DD0C00E01016615D8
:10665600016E6751080B026E0250080A02E1800EB5
:10666600011820E152C1E1FF53C1E2FF300EE66E90
:1066760050C100F051C101F037EC0EF0010166ABDC
:1066860003D0580E606F02D0780E606F52C1E1FFE2
:1066960053C1E2FF60C1E6FF50C100F051C101F0F5
:1066A60037EC0EF0800E006E800E01016219005C60
:1066B60002E16151635D0DE252C1E1FF53C1E2FFA8
:1066C600300EE66E50C100F051C101F037EC0EF00D
:1066D600E9D761C100F062C101F0010E0101615FFD
:1066E600000E625B00500110D8B42CD1C00E6615A6
:1066F600006E00C074F10AD161C100F062C101F000
:10670600000E62BFFF0E026E036E00360090013669
:106716000236033600360090013602360336010E85
:106726000024F66E8C0E0120F76E000E0220F86E25
:106736000900F5CF04F00900F5CF05F00900F5CF03
:1067460006F00900F5CF07F06EC100F06FC101F049
:1067560070C102F071C103F0FCEC04F00A0E046E85
:10676600000E056E066E076EFCEC04F008C000F025
:1067760009C001F00AC002F00BC003F0300E00247D
:10678600636FD3D066AB45D061C100F062C101F042
:10679600000E62BFFF0E026E036E003600900136D9
:1067A6000236033600360090013602360336290ECD
:1067B6000024F66E8D0E0120F76E000E0220F86E94
:1067C6000900F5CF04F00900F5CF05F00900F5CF73
:1067D60006F00900F5CF07F06EC100F06FC101F0B9
:1067E60070C102F071C103F0FCEC04F00F0E00164C
:1067F600000E011602160316C00E0024F66E8E0E4B
:106806000120F76E000E0220F86E0900F5CF63F145
:1068160044D061C100F062C101F0000E62BFFF0EFC
:10682600026E036E003600900136023603360036DD
:106836000090013602360336290E0024F66E8D0EC0
:106846000120F76E000E0220F86E0900F5CF04F065
:106856000900F5CF05F00900F5CF06F00900F5CFE0
:1068660007F06EC100F06FC101F070C102F071C196
:1068760003F0FCEC04F00F0E0016000E01160216D3
:1068860003169E0E0024F66E8E0E0120F76E000E85
:106896000220F86E0900F5CF63F147D061C100F020
:1068A60062C101F0000E62BFFF0E026E036E00367B
:1068B6000090013602360336003600900136023665
:1068C6000336A10E0024F66E8B0E0120F76E000E25
:1068D6000220F86E0900F5CF04F00900F5CF05F0A7
:1068E6000900F5CF06F00900F5CF07F06EC100F0FC
:1068F6006FC101F070C102F071C103F0FCEC04F04D
:10690600070E0014636F300E63270FD07451000A10
:10691600D8B4F2D67451C00AD8B4EED67451800AEF
:10692600D8B430D77451400AB9E052C1E1FF53C11F
:10693600E2FF63C1E6FF50C100F051C101F037EC40
:106946000EF0C7D6010166A71DD0800E006E800E20
:106956006519005C02E16451000814E252C1E1FFCE
:1069660053C1E2FF200EE66E50C100F051C101F0A6
:1069760037EC0EF0010E0101645F000E655B645199
:106986006511ECE130EF24F072C100F073C101F043
:026996001200ED
:1069980001015251531108E052C1E1FF53C1E2FF16
:1069A80050C1E6FF51C1E6FF50C1E9FF51C1EAFFFE
:1069B800EECF00F000C056F100C07AF1A2EC12F060
:1069C800005203E0504B512BEFD7546B000E56BFCB
:1069D800FF0E006E000E001802E12D0E561905E19B
:1069E800010E546F504B512B0CD0000E56BFFF0EAA
:1069F800006E000E001802E12B0E561902E1504BF2
:106A0800512B566B576B586B596B5A6B556B54B966
:106A18000BD050C1E9FF51C1EAFFEE502E0A04E144
:106A28005489504B512B54D050C1E9FF51C1EAFF52
:106A3800EECFA2F199EC07F0005201E14AD054835D
:106A48005651080A40E054A901D05507562B57C1A2
:106A580000F058C101F059C102F05AC103F00A0E02
:106A6800046E000E056E066E076EB2EC12F000C0E2
:106A780057F101C058F102C059F103C05AF10000A2
:106A8800000050C1E9FF51C1EAFF300EEE5C006E14
:106A9800016A000E015A000E01BEFF0E026E036E5F
:106AA8005751002658510122595102225A510322A6
:106AB80000C057F101C058F102C059F103C05AF1A2
:106AC8000000000003D054B901D0552B504B512B76
:106AD8009ED7566B50C1E9FF51C1EAFFEE50650AD7
:106AE80008E050C1E9FF51C1EAFFEE50450A01E054
:106AF80068D0504B512B50C1E9FF51C1EAFFEE500D
:106B08002D0A04E15487504B512B09D050C1E9FF9D
:106B180051C1EAFFEE502B0A02E1504B512B50C1F4
:106B2800E9FF51C1EAFFEE50300A03E1504B512B07
:106B3800F6D750C1E9FF51C1EAFFEECFA2F199ECB7
:106B480007F0005239E050C1E9FF51C1EAFF300EA9
:106B5800EE5C566F504B512B50C1E9FF51C1EAFF13
:106B6800EECFA2F199EC07F0005226E00A0E560388
:106B7800F3CF56F150C1E9FF51C1EAFF300EEE5C88
:106B8800006E00505627504B512B50C1E9FF51C1A0
:106B9800EAFFEECFA2F199EC07F000520DE00A0EE1
:106BA8005603F3CF56F150C1E9FF51C1EAFF300E49
:106BB800EE5C006E0050562754A703D056510008CB
:106BC800566F56515527000E531902E1000E5219FF
:106BD8000AE054A308D052C1E1FF53C1E2FF50C1FB
:106BE800E6FF51C1E6FF57C100F058C101F059C195
:106BF80002F05AC103F0F0EC22F000C057F101C0D6
:106C080058F102C059F103C05AF1046A056A066ACC
:106C1800076A57C100F058C101F059C102F05AC1C2
:106C280003F03DEC0DF0010ED8A4000E006E0052EA
:106C380005E0006A016A026A036A04D1800E5519E8
:106C4800006E800E000A005CD8B073D05551000861
:106C5800556F800E5519006E800E0A0A005C1DE300
:106C680057C100F058C101F059C102F05AC103F0F0
:106C7800FF0E046EE60E056E5B0E066E5D0E076E69
:106C8800BCEC01F000C057F101C058F102C059F145
:106C980003C05AF10A0E555FDCD75551000A1CE0B3
:106CA80057C100F058C101F059C102F05AC103F0B0
:106CB800CD0E046ECC0E056E4C0E066E7B0E076E66
:106CC800BCEC01F000C057F101C058F102C059F105
:106CD80003C05AF15507E1D7010E046E000E056E88
:106CE800000E066E010E076E57C100F058C101F084
:106CF80059C102F05AC103F09AEC06F0010ED8B05F
:106D0800000E006E005214E054A109D0010E006E6E
:106D1800000E016E800E026E030E036E93D0010EFC
:106D2800006E000E016E000E026E010E036E8AD018
:106D380072D0800E000A006E800E5519005C6BE25E
:106D48000A0E555D1DE357C100F058C101F059C145
:106D580002F05AC103F0F90E046E020E056E150E0C
:106D6800066EA00E076EBCEC01F000C057F101C022
:106D780058F102C059F103C05AF10A0E555FE0D725
:106D88005551000A1CE057C100F058C101F059C123
:106D980002F05AC103F0000E046E000E056E200EBC
:106DA800066E820E076EBCEC01F000C057F101C000
:106DB80058F102C059F103C05AF15507E1D757C13C
:106DC80004F058C105F059C106F05AC107F0FF0E8A
:106DD800006EFF0E016E7F0E026EFF0E036E9AECC0
:106DE80006F0010ED8B0000E006E005214E054A157
:106DF80009D0FF0E006EFF0E016EFF0E026EFF0E31
:106E0800036E20D0FF0E006EFF0E016E7F0E026E25
:106E1800FF0E036E17D054A10DD0000E5719006E47
:106E2800000E5819016E800E5919026E000E5A197B
:106E3800036E08D057C100F058C101F059C102F0E3
:066E48005AC103F0120024
:106E4E000B6A0350D8B46DEF37F002500A6E028E03
:106E5E008E0E035E03AE71EF37F0036C080E035C0B
:106E6E00D8A04CEF37F0036E013602C001F0026A73
:106E7E00080E035CD8A04CEF37F0036E0136016AA2
:106E8E000350D8A4D89056EF37F00350D8B456EF2D
:106E9E0037F0D89002320132032E50EF37F00BBC90
:106EAE0001A063EF37F0D8A063EF37F0012AD8B412
:106EBE00022A02BE80EF37F00AAE86EF37F0021ECE
:106ECE00011E012AD8B4022A86EF37F0026A016A3F
:106EDE0086EF37F00B800BAE8AEF37F0026A0AAE00
:106EEE008AEF37F0FF0E026E016E0A3602328AEF1B
:106EFE0037F0010E0C6EBBEC04F08CEF37F0000E89
:106F0E000C6E8CEF37F0FF0E0C6E0150006E0250BF
:046F1E00016E1200EE
:106F22009E9650C1C9FFC7A401D0FDD79EB601D01D
:106F3200FDD7C5BC02D0006A03D0C584020E006E24
:026F420012003B
:106F4400550E01015B6F010E5C6F50C17AF151C1A6
:106F54007BF152C17CF153C17DF154C17EF15B0ED2
:106F64007F6F010E806FDBEC12F000C059F101C09D
:106F74005AF100505025E16E01505121E26EE66A4B
:0A6F840059C100F05AC101F01200DB
:106F8E00A69C51C1AAFF50C1A9FFA69EA680A8CF5C
:046F9E0000F01200ED
:106FA2000D0E0101A76FC9EC04F00A0E0101A76FD3
:066FB200C9EC04F012001E
:106FB8000101536B50C1E9FF51C1EAFFEECF52F115
:106FC8005251000A0FE052C1A7F1C9EC04F00101C7
:106FD800532B53515025E96E000E5121EA6EEECF26
:066FE80052F1EED7120089
:106FEE000101506B516B5151120802E150518E0844
:106FFE0009E312EC23F0005201E004D00101504BE2
:10700E00512BF1D70101120E515D02E18F0E505D31
:10701E0003E37B0E006E05D0C580C5A001D0FDD761
:04702E00006A1200E2
:107032000B6A0C6A0A6A0350D8B44EEF38F00A9E03
:10704200028E860E035E03BE2CEF38F0D8B42CEF0E
:1070520038F051EF38F0036C080E035CD8A03AEF19
:1070620038F0036E0236026A0350D8A4D89043EF78
:1070720038F00350D8B443EF38F0D8900232032EE0
:107082003EEF38F00BBC02A04EEF38F0D8A04EEF26
:1070920038F0022AD8B458EF38F0016A5EEF38F0BF
:1070A2000B800BAE62EF38F0016A62EF38F0010E2E
:1070B2000C6EBBEC04F064EF38F0000E0C6E64EF63
:0C70C20038F0FF0E0C6E0250006E120041
:1070CE00800E0101516F5151000814E251515015BB
:1070DE00016E0150000805E2310EA76FC9EC04F0F5
:1070EE0005D0300E0101A76FC9EC04F00101513338
:0670FE00519FE9D71200CA
:1071040050C1F6FF51C1F7FF52C1F8FF0900F5CF96
:1071140000F0005212E050C1F6FF51C1F7FF52C116
:10712400F8FF0900F5CFA7F1C9EC04F0010E010145
:0C7134005027000E51235223E3D7120015
:10714000F00E01015015026E02C000F00032009EE8
:107150000032009E0032009E0032009E300E00245D
:10716000016E01C051F10150390802E2070E5127AA
:107170000F0E5015006E300E0024016E01C052F14A
:107180000150390802E2070E522751C1A7F1C9EC9C
:1071900004F052C1A7F1C9EC04F0680E0101A76F19
:0671A000C9EC04F012002E
:1071A6009E96C5869EB601D0FDD7C9CF01F00101D6
:1071B6005051000A02E1C58A01D0C59A9E96C5883B
:0C71C6009EB601D0FDD701C000F0120001
:0471D200C58412005E
:0A71D600C582C5A201D0FDD712004A
:1071E00000C008F00150006E016A026A036A0B6A6F
:1071F0000C6A016A026A036A960E036E0A6A00AE9E
:1072000008EF39F0081E001E082AD8B4002A0A8E9A
:1072100000C001F008C000F0086A026AFBEC0DF043
:0272200012005A
:10722200920E0101316F090E326FA70E336F010EFC
:10723200346FFF0E256FFF0E266F000E276F000EB4
:10724200286FFF0E296FFF0E2A6F000E2B6F000EA4
:107252002C6FFF0E2D6FFF0E2E6F000E2F6F000E84
:10726200306FAC8A900EAB6E948E949C9EAA03D023
:08727200AECF00F0FBD71200C3
:10727A0039C13BF13AC13CF13BC150F13CC151F13A
:10728A0081DE00C03DF1000E01013E6F000E3E1985
:10729A0002E1000E3D1901E12FD0800E030A006EB3
:1072AA00800E3C19005C02E13B51FF0801E224D048
:1072BA003DC1A7F1C9EC04F0010139513B5D006EF3
:1072CA003A513C59016EB00E0024E16E000E0120C5
:1072DA00E26E3DC1E6FF210E0C6E760E0D6E0D2E8E
:1072EA00FED70C2EFCD700003B4B3C2B000E3E1960
:0A72FA0002E1000E3D19C0E1120090
:107304000900F5CFE6FF0006FBE10106F9E11200F2
:10731400FF0E816E0F01396BFF0E936E2F0E806E80
:10732400386B388138832F0E926E806A826A3A6B8A
:10733400FF0E946E94869488948E949C606A1200D6
:10734400400E0101416F010E426F39C150F13AC143
:1073540051F13BC152F13CC153F13DC154F13EC125
:1073640055F13FC156F1410E576F010E586F2BEC8A
:0473740024F01200EF
:107378003BC1F6FF3CC1F7FF3DC1F8FF0900F5CF5F
:1073880000F0005218E03BC1F6FF3CC1F7FF3DC1D9
:10739800F8FF0900F5CF00F039C1E1FF3AC1E2FF7B
:1073A80000C0E6FF0101394B3A2B010E3B27000EC6
:1073B8003C233D23DDD739C1E1FF3AC1E2FFE66A4C
:0273C8001200B1
:1073CA0011DE900E0101506FA7DD110E0C6E3A0E00
:1073DA000D6E0D2EFED70C2EFCD70000510E0101AA
:0873EA00506F9ADDF1DE120084
:1073F200FDDD900E0101506F93DDA20E0101506F71
:107402008FDD110E0C6E3A0E0D6E0D2EFED70C2E68
:10741200FCD70000EBDD910E0101506F81DD110EF2
:107422000C6E3A0E0D6E0D2EFED70C2EFCD7000000
:10743200010E0101506FB6DE00C035F0110E0C6E68
:107442003A0E0D6E0D2EFED70C2EFCD70000010158
:10745200506BA8DE00C034F0BBDE36C050F137C03E
:1074620051F1E80E0101526F8C0E536F000E546FF2
:1074720035C055F1000E566F34C057F1000E586FEB
:0E74820060DD36C050F137C051F195DD1200CB
:1074900001013F51000805E3070E406F000E416FE8
:1074A00012D03F51160805E2170E426F000E436FCF
:1074B00006D03F51010F426F436B000E432342C180
:1074C00040F143C141F140C14AF141C14BF1446B2C
:1074D000456B046A056A066A076A39C100F03AC159
:1074E00001F03BC102F03CC103F09AEC06F0010E42
:1074F000D8B0000E006E005209E03DC1E1FF3EC170
:10750000E2FF2D0EE66E3D4B3E2B3B7F39C104F072
:107510003AC105F03BC106F03CC107F0006A016AC0
:10752000026A036A9AEC06F0010ED8B0000E006EF3
:10753000005237E0000E046E000E056E000E066E5F
:107540007F0E076E39C100F03AC101F03BC102F075
:107550003CC103F09AEC06F0010ED8B0000E006EAC
:1075600000521FE039C100F03AC101F03BC102F006
:107570003CC103F0000E046E000E056E200E066E78
:10758000820E076EBCEC01F000C039F101C03AF187
:1075900002C03BF103C03CF1010E445F000E455BAD
:1075A000C9D7000E046E000E056E200E066E820E08
:1075B000076E39C100F03AC101F03BC102F03CC195
:1075C00003F09AEC06F0000ED8B0010E006E0052E7
:1075D0001EE0000E046E000E056E200E066E820E7A
:1075E000076E39C100F03AC101F03BC102F03CC165
:1075F00003F08EEC09F000C039F101C03AF102C08D
:107600003BF103C03CF10101444B452BCAD7445127
:107610004A2745514B23010E466F000E476F010E5E
:10762000006E000E016EDCDD00C04CF101C04DF1BA
:1076300002C04EF103C04FF1800E4719006E800E5C
:107640004B19005C02E14A51465D1EE2000E046ED9
:10765000000E056E200E066E820E076E4CC100F005
:107660004DC101F04EC102F04FC103F08EEC09F0A4
:1076700000C04CF101C04DF102C04EF103C04FF10A
:107680000101464B472BD8D7000E046E000E056E45
:10769000000E066E800E076E4CC100F04DC101F069
:1076A0004EC102F04FC103F08EEC09F039C104F075
:1076B0003AC105F03BC106F03CC107F0AAEC02F06C
:1076C00000C039F101C03AF102C03BF103C03CF106
:1076D000000E046E000E056E200E066E820E076E02
:1076E0009AEC06F0000ED8B0010E006E00520BE0CE
:1076F000000E0101396F000E3A6F000E3B6F7F0ED6
:107700003C6F444B452B0101800E4519006E800EE5
:10771000005C02E1000E445D38E23DC1E1FF3EC184
:10772000E2FF300EE66E3D4B3E2B3DC1E1FF3EC118
:10773000E2FF2E0EE66E3D4B3E2B800E4B19006E87
:10774000800E005C02E1000E4A5D04E24A51445F93
:107750004B51455BFF0E466FFF0E476F800E45197C
:10776000006E800E4719005C02E14651445D0DE257
:107770003DC1E1FF3EC1E2FF300EE66E3D4B3E2BC8
:10778000010E465F000E475BE9D7466B476B800EE4
:107790004719006E800E4B19005C02E14A51465DAC
:1077A00062E239C100F03AC101F03BC102F03CC1D4
:1077B00003F027EC37F000C048F101C049F1300E6A
:1077C00000263DC1E1FF3EC1E2FF00C0E6FF3D4BA8
:1077D0003E2B4751451902E14451461908E13DC18C
:1077E000E1FF3EC1E2FF2E0EE66E3D4B3E2B48C14F
:1077F00000F049C101F0F4DC00C04CF101C04DF1D2
:1078000002C04EF103C04FF100C004F001C005F00A
:1078100002C006F003C007F039C100F03AC101F020
:107820003BC102F03CC103F026EC09F000C039F185
:1078300001C03AF102C03BF103C03CF1000E046EFE
:10784000000E056E200E066E820E076EBCEC01F077
:1078500000C039F101C03AF102C03BF103C03CF174
:10786000464B472B94D73DC1E1FF3EC1E2FFE66A9C
:02787000120004
:10787200F7EC37F0900E0101506F91EC37F0AA0E41
:107882000101506F91EC37F0110E0C6E3A0E0D6E35
:107892000D2EFED70C2EFCD700009CDC910E0101B0
:1078A200506F91EC37F0110E0C6E3A0E0D6E0D2EDC
:1078B200FED70C2EFCD70000010E0101506F72DCC6
:1078C20000C039F0110E0C6E3A0E0D6E0D2EFED761
:1078D2000C2EFCD700000101506B64DC00C038F0B4
:1078E200110E0C6E3A0E0D6E0D2EFED70C2EFCD71D
:1078F20000006EDC39507F0804E2010E326E000E89
:10790200336E7F0E3914006E00C039F036C050F16C
:1079120037C051F19E0E0101526F8C0E536F000E53
:10792200546F00C055F1000E566F38C057F1000E6B
:10793200586FA2EC37F036C050F137C051F1DCEC91
:0479420037F0120008
:1079460039C150F13AC151F13BC152F13CC153F139
:107956001FEC23F000C004F001C005F002C006F0E1
:1079660003C007F039C100F03AC101F03BC102F093
:107976003CC103F026EC09F0000E046E400E056EC5
:107986001C0E066E8C0E076EBCEC01F054EC0DF06E
:1079960000C03EF101C03FF102C040F103C041F119
:1079A60000C050F101C051F102C052F103C053F1C1
:1079B60036C054F137C055F1BAEC23F036C050F159
:1079C60037C051F1DCEC37F0090EA76FC9EC04F0B3
:1079D600090E0101A76FC9EC04F039C150F13AC193
:1079E60051F13BC152F13CC153F11FEC23F019ECAC
:1079F60038F000C000F100C050F1A0EC38F0090EDC
:107A06000101A76FC9EC04F001013D6B000E415D59
:107A160008E1000E405D05E1130E3F5D02E1880EB0
:107A26003E5D0AE3800E3D27880E3E5F130E3F5BE8
:107A3600000E405B000E415B000E415D08E1000E4A
:107A4600405D05E1090E3F5D02E1C40E3E5D0AE3BD
:107A5600400E3D27C40E3E5F090E3F5B000E405BA5
:107A6600000E415B000E415D08E1000E405D05E140
:107A7600040E3F5D02E1E20E3E5D0AE3200E3D2765
:107A8600E20E3E5F040E3F5B000E405B000E415B64
:107A9600000E415D08E1000E405D05E1020E3F5D0E
:107AA60002E1710E3E5D02E3100E3D273DC150F12D
:107AB600A0EC38F0090E0101A76FC9EC04F0F7EC51
:107AC60037F0900E0101506F91EC37F0110E0C6EED
:107AD6003A0E0D6E0D2EFED70C2EFCD70000A10E11
:107AE6000101506F91EC37F0110E0C6E3A0E0D6ECF
:107AF6000D2EFED70C2EFCD7000000C150F191ECE4
:107B060037F03DC150F191EC37F0110E0C6E3A0E84
:107B16000D6E0D2EFED70C2EFCD70000E9EC38F0CA
:107B260036C050F137C051F1510E0101526F8C0E23
:107B3600536F000E546F00C155F1000E566F3DC1D4
:107B460057F1000E586FA2EC37F036C050F137C02F
:087B560051F1DCEC37F01200E4
:107B5E0039C150F13AC151F10101526B536BCCEC6A
:047B6E0034F01200DD
:107B7200F7EC37F0900E0101506F91EC37F0110ED7
:107B82000C6E3A0E0D6E0D2EFED70C2EFCD7000099
:107B9200220E0101506F91EC37F0E9EC38F012003F
:107BA20039C150F13AC151F13BC152F13CC153F1DB
:107BB2001FEC23F000C004F001C005F002C006F083
:107BC20003C007F039C100F03AC101F03BC102F035
:107BD2003CC103F026EC09F0000E046E400E056E67
:107BE2001C0E066E8C0E076EBCEC01F054EC0DF010
:107BF20000C03EF101C03FF102C040F103C041F1BB
:107C020000C050F101C051F102C052F103C053F162
:107C120036C054F137C055F1BAEC23F036C050F1FA
:107C220037C051F1DCEC37F0090EA76FC9EC04F054
:107C3200090E0101A76FC9EC04F039C150F13AC134
:107C420051F13BC152F13CC153F11FEC23F019EC4D
:107C520038F000C000F100C050F1A0EC38F0090E7D
:107C62000101A76FC9EC04F001013D6B000E415DFB
:107C720008E1000E405D05E1130E3F5D02E1880E52
:107C82003E5D0AE3800E3D27880E3E5F130E3F5B8A
:107C9200000E405B000E415B000E415D08E1000EEC
:107CA200405D05E1090E3F5D02E1C40E3E5D0AE35F
:107CB200400E3D27C40E3E5F090E3F5B000E405B47
:107CC200000E415B000E415D08E1000E405D05E1E2
:107CD200040E3F5D02E1E20E3E5D0AE3200E3D2707
:107CE200E20E3E5F040E3F5B000E405B000E415B06
:107CF200000E415D08E1000E405D05E1020E3F5DB0
:107D020002E1710E3E5D02E3100E3D273DC150F1CE
:107D1200A0EC38F0090E0101A76FC9EC04F0F7ECF2
:107D220037F0900E0101506F91EC37F0A20E010175
:107D3200506F91EC37F0110E0C6E3A0E0D6E0D2E47
:107D4200FED70C2EFCD7000000C150F191EC37F0A9
:107D5200110E0C6E3A0E0D6E0D2EFED70C2EFCD7A8
:107D620000003DC150F191EC37F0110E0C6E3A0E4D
:107D72000D6E0D2EFED70C2EFCD70000E9EC38F06C
:107D820036C050F137C051F1780E0101526F8C0E9E
:107D9200536F000E546F00C155F1000E566F3DC176
:107DA20057F1000E586FA2EC37F036C050F137C0D1
:087DB20051F1DCEC37F0120086
:107DBA00F7EC37F000C150F191EC37F0005216E0C1
:107DCA0036C050F137C051F1C30E0101526F8C0E0B
:107DDA00536F000E546F00C155F1A2EC37F036C054
:107DEA0050F137C051F1DCEC37F015D0010136C043
:107DFA0050F137C051F1490E526F8D0E536F000E7C
:107E0A00546F00C155F1A2EC37F036C050F137C0BB
:107E1A0051F1DCEC37F0E9EC38F0D1EC37F0120034
:107E2A00949894968B988B9694889486C79EC79CB0
:067E3A00380EC66E1200B6
:107E4000F7EC37F0900E0101506F91EC37F0540EC3
:0E7E50000101506F91EC37F0E9EC38F01200B0
:107E5E00F7EC37F0900E0101506F91EC37F0A10E58
:107E6E000101506F91EC37F0F7EC37F0910E0101F4
:107E7E00506F91EC37F0110E0C6E3A0E0D6E0D2EFA
:107E8E00FED70C2EFCD70000010E0101506FD3EC73
:107E9E0038F000C02CF0110E0C6E3A0E0D6E0D2E39
:107EAE00FED70C2EFCD700000101506BD3EC38F03E
:107EBE0000C02BF0E9EC38F036C050F137C051F16C
:107ECE00690E0101526F8D0E536F000E546F2CC050
:107EDE0055F1000E566F2BC057F1000E586FA2ECE5
:107EEE0037F036C050F137C051F1DCEC37F01200EC
:107EFE00F7EC37F0900E0101506F91EC37F0AC0EAD
:107F0E000101506F91EC37F0110E0C6E3A0E0D6EA2
:107F1E000D2EFED70C2EFCD70000EBEC38F0910E98
:107F2E000101506F91EC37F0110E0C6E3A0E0D6E82
:107F3E000D2EFED70C2EFCD700000101506BD3EC9A
:107F4E0038F000C02DF0E9EC38F0F00E0101506F62
:107F5E008E0E516F000E526F82EC38F02DC050F124
:107F6E00A0EC38F0090E0101A76FC9EC04F02DC08A
:0C7F7E0050F167EC38F0D1EC37F0120045
:107F8A00F7EC37F0900E0101506F91EC37F0AC0E20
:107F9A000101506F91EC37F0110E0C6E3A0E0D6E16
:107FAA000D2EFED70C2EFCD7000000C150F191EC2B
:087FBA0037F0E9EC38F0120089
:107FC2007FEC47F08AEC39F0B886010EB06E030EF2
:107FD200AF6EAC8411EC39F0020E0B6E450E0C6ED6
:107FE200A90E0D6E0D2EFED70C2EFCD70B2EFAD736
:107FF200000000000C0EA76FC9EC04F0070E0B6E18
:10800200580E0C6E590E0D6E0D2EFED70C2EFCD78F
:108012000B2EFAD700000000306A316A2E6A2F6AEE
:108022003A0E366E000E376E36C039F137C03AF16D
:10803200260E01013B6F8A0E3C6F000E3D6FBCECB9
:1080420039F036C050F137C051F1DCEC37F0A30EF5
:108052000C6E550E0D6E0D2EFED70C2EFCD736C0B3
:1080620039F137C03AF1D80E3B6F890E3C6F000EE2
:108072003D6FBCEC39F036C050F137C051F1DCEC49
:1080820037F0E00E396F1B0E3A6FA20E3B6F010EF6
:108092003C6FC50E3D6F8D0E3E6F000E3F6FA2EC22
:1080A20039F00D0E0B6EAF0E0C6EB60E0D6E0D2E60
:1080B200FED70C2EFCD70B2EFAD700003A6A3A0EE6
:1080C200366E000E376EE00E396F1B0E3A6FA20E3F
:1080D2003B6F010E3C6F7B0E3D6F8E0E3E6F000EAE
:1080E2003F6FA2EC39F0396B3A6B3DEC39F0200E60
:1080F200396F000E3A6F3DEC39F036C050F137C09F
:1081020051F1FB0E526F8D0E536F000E546FA2ECA5
:1081120037F036C050F137C051F1DCEC37F0190EB0
:10812200C86E82DE800E396F000E3A6F3DEC39F078
:10813200D1EC37F0900E0101006F3EDED1EC37F04A
:10814200020E0B6E450E0C6EA90E0D6E0D2EFED795
:108152000C2EFCD70B2EFAD70000000070DE020EA8
:108162000B6E450E0C6EA90E0D6E0D2EFED70C2E4B
:10817200FCD70B2EFAD7000000000E0E0101006F93
:1081820003DF0D0E0B6EAF0E0C6EB60E0D6E0D2EC6
:10819200FED70C2EFCD70B2EFAD70000AFDE020E54
:1081A2000B6E450E0C6EA90E0D6E0D2EFED70C2E0B
:1081B200FCD70B2EFAD70000000050DE2BC005F0D2
:1081C200000E066E076E086E040E046E05C000F007
:1081D20006C001F007C002F008C003F0045009E035
:1081E2000332023201320032039E03BC038EFF0FC0
:1081F200F6D700C0D4F001C0D5F002C0D6F003C05B
:10820200D7F03E0E046E000E056E000E066E000ED6
:10821200076EB2EC12F000C0D4F001C0D5F002C07B
:10822200D6F003C0D7F02CC000F0000E016E026E33
:10823200036EE80E046E030E056E000E066E076EE8
:10824200B2EC12F00001D4510026D5510122D651D0
:108252000222D751032200C0D4F001C0D5F002C0DF
:10826200D6F003C0D7F0F0EC22F0000E046E000E40
:10827200056E7A0E066E880E076E8EEC09F000C04F
:10828200D0F001C0D1F002C0D2F003C0D3F000C0E0
:1082920039F101C03AF102C03BF103C03CF1D80E02
:1082A20001013D6F000E3E6F030E3F6F48EC3AF046
:1082B20036C050F137C051F1140E526F8E0E536F0B
:1082C200000E546FD80E556F000E566FA2EC37F0A9
:1082D20036C050F137C051F1DCEC37F0020E0B6EB4
:1082E200450E0C6EA90E0D6E0D2EFED70C2EFCD770
:1082F2000B2EFAD700000000F9EC39F034C005F07B
:10830200000E066E076E086E040E046E05C000F0C5
:1083120006C001F007C002F008C003F0045009E0F3
:108322000332023201320032039E03BC038EFF0F7E
:10833200F6D700C0D4F001C0D5F002C0D6F003C019
:10834200D7F03E0E046E000E056E000E066E000E95
:10835200076EB2EC12F000C0D4F001C0D5F002C03A
:10836200D6F003C0D7F035C000F0000E016E026EE9
:10837200036EE80E046E030E056E000E066E076EA7
:10838200B2EC12F00001D4510026D5510122D6518F
:108392000222D751032200C0D4F001C0D5F002C09E
:1083A200D6F003C0D7F0F0EC22F0000E046E000EFF
:1083B200056E7A0E066E880E076E8EEC09F000C00E
:1083C200D0F001C0D1F002C0D2F003C0D3F000C09F
:1083D20039F101C03AF102C03BF103C03CF1D80EC1
:1083E20001013D6F000E3E6F030E3F6F48EC3AF005
:1083F20036C050F137C051F1400E526F8E0E536F9E
:10840200000E546FD80E556F000E566FA2EC37F067
:1084120036C050F137C051F1DCEC37F0D1EC37F017
:10842200020E0B6E450E0C6EA90E0D6E0D2EFED7B2
:108432000C2EFCD70B2EFAD700000000E5EC39F029
:108442000A0E0B6E840E0C6E070E0D6E0D2EFED7ED
:108452000C2EFCD70B2EFAD700000000D1EC37F01F
:108462000001FA6BFB6BF86BF96BAB8ED08EF28C62
:108472009D8AA39A9E9AF28E3A0E366E000E376E3F
:1084820039EC3CF038C005F0000E066E076E086E3F
:10849200040E046E05C000F006C001F007C002F031
:1084A20008C003F0045009E0033202320132003204
:1084B200039E03BC038EFF0FF6D700C0D4F001C0A9
:1084C200D5F002C0D6F003C0D7F0710E046E020ED2
:1084D200056E000E066E000E076EB2EC12F000C0C2
:1084E200D4F001C0D5F002C0D6F003C0D7F039C035
:1084F20000F0000E016E026E036E100E046E270E67
:10850200056E000E066E076EB2EC12F00001D45139
:108512000026D5510122D6510222D751032200C092
:10852200D4F001C0D5F002C0D6F003C0D7F0F0EC11
:1085320022F0000E046E400E056E1C0E066E8C0EAE
:10854200076E8EEC09F000C0D0F001C0D1F002C07D
:10855200D2F003C0D3F000C039F101C03AF102C039
:108562003BF103C03CF1D80E01013D6F000E3E6F9E
:10857200030E3F6F48EC3AF036C050F137C051F16C
:108582002A0E526F8E0E536F000E546FD80E556F17
:10859200000E566FA2EC37F036C050F137C051F1E1
:1085A200DCEC37F0000E0001FB1902E1010EFA19B2
:1085B200D8A4CAD1B9EC3DF036C050F137C051F160
:1085C200E10E0101526F8E0E536F000E546FA2EC3A
:1085D20037F036C050F137C051F1DCEC37F0980E6D
:1085E200506F000E516FDCEC37F0D1EC37F0000128
:1085F2009851480AD8A490D0800E006E800E971928
:10860200005C02E196510508D8B086D0990E0101AE
:10861200396F000E3A6FAFEC3DF000C092F001C02E
:1086220093F002C094F003C095F000C004F001C0C2
:1086320005F002C006F003C007F08AC000F08BC04C
:1086420001F08CC002F08DC003F09AEC06F0010E2E
:10865200D8B0000E006E005239E092C08EF093C086
:108662008FF094C090F095C091F092C039F193C010
:108672003AF194C03BF195C03CF1D80E3D6F000E2B
:108682003E6F020E3F6F48EC3AF036C050F137C0F1
:1086920051F1A90E526F8D0E536F000E546FD80E0A
:1086A200556F000E566FA2EC37F036C050F137C04E
:1086B20051F1DCEC37F08EC039F18FC03AF190C045
:1086C2003BF191C03CF1A3EC3CF026D08AC039F1D9
:1086D2008BC03AF18CC03BF18DC03CF1D80E3D6F9E
:1086E200000E3E6F020E3F6F48EC3AF036C050F17A
:1086F20037C051F19C0E526F8A0E536F000E546FA9
:10870200D80E556F000E566FA2EC37F036C050F1FE
:1087120037C051F1DCEC37F000019851420AD8A47D
:10872200F9D0800E006E800E9719005C02E196511E
:108732000508D8B0EFD0990E0101396F000E3A6FDB
:10874200AFEC3DF000C035F101C036F102C037F1A7
:1087520003C038F135C192F036C193F037C194F0BD
:1087620038C195F08EC000F08FC001F090C002F0C9
:1087720091C003F0000E046E000E056E000E066E30
:108782007F0E076EAAEC02F000C004F001C005F0F3
:1087920002C006F003C007F035C100F036C101F097
:1087A20037C102F038C103F09AEC06F0010ED8B0DE
:1087B200000E006E005239E092C08AF093C08BF036
:1087C20094C08CF095C08DF092C039F193C03AF10B
:1087D20094C03BF195C03CF1D80E3D6F000E3E6F48
:1087E200020E3F6F48EC3AF036C050F137C051F1FB
:1087F200E00E526F8D0E536F000E546FD80E556FF0
:10880200000E566FA2EC37F036C050F137C051F16E
:10881200DCEC37F08AC039F18BC03AF18CC03BF105
:108822008DC03CF1D1EC3DF026D08EC039F18FC025
:108832003AF190C03BF191C03CF1D80E3D6F000E71
:108842003E6F020E3F6F48EC3AF036C050F137C02F
:1088520051F1660E526F8A0E536F000E546FD80E8E
:10886200556F000E566FA2EC37F036C050F137C08C
:1088720051F1DCEC37F000019851430A4BE1995178
:10888200460A48E19A51470A45E1800E006E800E81
:108892009719005C02E1965103083CE2B9EC3DF005
:1088A20036C050F137C051F1550E0101526F8E0E94
:1088B200536F000E546FA2EC37F036C050F137C040
:1088C20051F1DCEC37F020EC3FF036C050F137C00C
:1088D20051F1D10E0101526F8E0E536F000E546F83
:1088E200A2EC37F036C050F137C051F1DCEC37F072
:1088F200020E0B6E450E0C6EA90E0D6E0D2EFED7DE
:108902000C2EFCD70B2EFAD7000000000E0E006FC3
:10891200C5EC3FF00001FA6BFB6B966B976B986BA3
:108922007FEC3FF0D1EC37F0020E0B6E450E0C6E71
:10893200A90E0D6E0D2EFED70C2EFCD70B2EFAD7DC
:1089420000000000E5EC39F0000E0001FB1902E125
:10895200020EFA1930E136C050F137C051F1090E5A
:108962000101526F8D0E536F000E546F180E556F2A
:10897200A2EC37F036C050F137C051F1DCEC37F0E1
:10898200980E506F000E516FDCEC37F0D1EC37F0DF
:10899200270E0B6E0D0E0C6E260E0D6E0D2EFED7D3
:1089A2000C2EFCD70B2EFAD700000001FA6BFB6BE2
:1089B200966B976B9D8A140E0B6E070E0C6E110E42
:1089C2000D6E0D2EFED70C2EFCD70B2EFAD7000003
:0689D200000052D5FFD7A2
:108EFE0010EE19F0120E006E010E016E690EF66E76
:0E8F0E008E0EF76E000EF86E82EC39F0120037
:1089D800433A5F4D696B726F435F4D657350726FB9
:1089E8006A6574735F4D696B726F435F31384632E5
:1089F800364B32325F4453313633310138463236E2
:108A08004B32325F4453313633315F74656D706574
:0E8A1800725F3135303332352E630A0D200087
:108A26004D696B726F632070726F20362E30312065
:108A36005465737420636170746575722064652073
:108A460074656D7065726174757265204453313654
:108A5600333120493243203135303332350A0D0067
:108A6600536575696C204861757420646F6974205C
:108A76006574726520696E666572696575722061D6
:108A86007520736575696C2068617574202573207F
:068A9600B043200D0A00B0
:108A9C00536575696C204861757420646F69742026
:108AAC006574726520737570657269657572206185
:108ABC007520736575696C2062617320257320B015
:058ACC0043200D0A002B
:108AD1000000007FCDCC4C7B0AD723786F12037541
:108AE10017B75171ACC5276EBD37066B95BF566779
:108AF10077CC2B645F700961FFE65B5D08E53C3C68
:048B01006042221B91
:108B05000000007F000020820000488500007A8870
:108B150000401C8C0050438F002474928096189658
:108B250020BC3E99286B6E9CF90215A0EC782DC1EE
:048B3500CAF249E255
:108B39000000007F000020820000488500007A883C
:108B490000401C8C0050438F002474928096189624
:108B590020BC3E99286B6E9CF90215A0EC782DC1BA
:048B6900CAF249E221
:108B6D000000007FCDCC4C7B0AD723786F120375A4
:108B7D0017B75171ACC5276EBD37066B95BF5667DC
:108B8D0077CC2B645F700961FFE65B5D08E53C3CCB
:048B9D006042221BF5
:108BA1000100000008000000400000000002000079
:108BB1000010000000800000000004000000200000
:108BC100000000010000000800000040000000005B
:108BD1000100000008000000400000000002000049
:108BE10000100000008000000000040000002000D0
:108BF100000000010000000800000040000000002B
:108C0100010000000A00000064000000E803000009
:108C110010270000A086010040420F0080969800B6
:088C210000E1F50500CA9A3BD1
:108C2900010000000A00000064000000E8030000E1
:108C390010270000A086010040420F00809698008E
:088C490000E1F50500CA9A3BA9
:108C51000D0A20496E697420536575696C2048615D
:108C610075742053313D25303258202053323D2533
:078C7100303258200D0A000B
:108C78000D0A20496E697420536575696C2042613C
:108C8800732053313D25303258202053323D253052
:068C98003258200D0A0015
:108C9E005261772054656D706572204453313633BE
:108CAE00312064483D253032582020644C3D25301B
:058CBE003258200900FE
:108CC30044657669636520617420616472657373BA
:108CD30065202530325820206973206E6F7420661A
:058CE3006F756E6400D6
:108CE80020536575696C20426173202053624820C7
:108CF8003D253032782053624C3D253032782009AA
:018D0800006A
:108D0900427566666572312046554C4C20212025F6
:108D19002033642063617273206D6178690D0A00E4
:108D29000100000010000000000100000010000018
:108D39000000010000001000000000010000001008
:108D49004465766963652061742061647265737333
:108D590065202530325820666F756E64204F4B00B0
:108D690020536575696C2048617574205368483DC6
:108D7900253032582053686C3D253032582009007F
:108D890001000000100000000001000000100000B8
:108D990000000100000010000000000100000010A8
:108DA9004D6F64696620536575696C2048617574F7
:0C8DB900206120257320B043200D0A002B
:108DC5004F7363696C6C617465757220517561725E
:0B8DD500747A3D31304D687A0D0A00C1
:108DE0004D6F64696620536575696C20426173201C
:0B8DF0006120257320B043200D0A0015
:108DFB0056657273696F6E203A203235206D617241
:098E0B007320323031350D0A00EC
:108E1400536575696C2048617574203D2025732065
:068E2400B043200D0A001E
:108E2A0054656D70657261747572653D2025732095
:068E3A00B043200D0A0008
:108E4000536575696C20626173203D20257320B0E5
:058E500043200D0A00A3
:108E550052656C65637475726520436F6E666967EC
:048E6500203D0900A3
:028E6900000007
:028E6B00000005
:078E6D00286E756C6C2900F2
:078E7400286E756C6C2900EB
:108E7B0050726573656E746174696F6E203A200D64
:028E8B000A00DB
:108E8D003031323334353637383961626364656673
:018E9D0000D4
:108E9E003031323334353637383961626364656662
:018EAE0000C3
:108EAF003031323334353637383941424344454611
:018EBF0000B2
:108EC0003031323334353637383941424344454600
:018ED00000A1
:108ED100536F66747761726520504F52200D0A00FE
:0F8EE1005265636570742055415254313D200035
:0D8EF0000D0A436F6E66696720634C3D00FC
:020000040030CA
:0D000100231F3CFFBF81FF0FC00FE00F4029
:0200000400F00A
:1000000031384632364B3232202031304D487A205A
:100010004D696B726F432056362E3530200D0A0025
:100020004453313633312054656D7065722E202073
:10003000204932432053656E736F720D0A00000031
:1000400020202020202020202020202020202020B0
:100050002E2E2E2E2E2E2E2E2E2E2E2E2E2E2E00EE
:100060005265736572766520202020202020202094
:10007000526573657276652020202020200D0A00CD
:10008000496E697420493243203130304B687A0D13
:100090000A00202020202020202020202020202096
:1000A000496E69742041444320200D0A000000007D
:1000B00056657269662054656D706F2044656C6189
:1000C0007920323030306D5320200D0A0000FFFFC0
:1000D000FFFFFFFFFFFFFFFFFFFFFFFFFFFFFF002F
:1000E000FFFFFFFFFFFFFFFFFFFFFFFFFFFFFFFF20
:1000F000FFFFFFFFFFFFFFFFFFFFFFFFFFFFFF000F
:10010000FFFFFFFFFFFFFFFFFFFFFFFFFFFFFFFFFF
:10011000FFFFFFFFFFFFFFFFFFFFFFFFFFFFFFFFEF
:10012000FFFFFFFFFFFFFFFFFFFFFFFFFFFFFFFFDF
:10013000FFFFFFFFFFFFFFFFFFFFFFFFFFFFFFFFCF
:1003F0007061756C666A756A6F0D0A00FFFFFFFF1A
:00000001FF
